:020000040000FA
:060000006CEF3FF012005E
:060800006CEF3FF0120056
:06082A000600B07F000093
:10083000E90100000C000000AF7F0000B5020000DD
:1008400001000000A97F0000FA000000060000007F
:10085000317F0000B4020000010000009C7F000016
:10086000DC0100000D000000987F0000AA020000DB
:040870000400000080
:0C08740004001200D9CFE6FFE1CFD9FF4D
:1008800081E945E8030E056E0101E551010A17E013
:10089000010A2AE10A0EE45D09E10001DA51016E64
:1008A000DB51026EDC51036EDD511DD0020100519F
:1008B000016E0151026E0251036E035114D00A0EF3
:1008C000E45D09E10001DE51016EDF51026EE0518D
:1008D000036EE15108D002010451016E0551026E10
:1008E0000651036E0751046E97EC0AF0030A2DE0DF
:1008F000070A1BE0010A0AE0050A04E0010A02E017
:10090000030A35E1810EE66E740E34D07C0EE66E7D
:10091000740E0DEC0AF00001CB51E66EE66A030E90
:10092000E66ECF0EE66E000E2CD0770EE66E740EDD
:100930000DEC0AF0DCC1E6FFDDC1E6FFDEC1E6FF3B
:10094000DFC1E6FF9BEC0AF017D0720EE66E740E64
:100950000DEC0AF0E0C1E6FFE1C1E6FFE2C1E6FF0F
:10096000E3C1E6FF9BEC0AF0040E056E05D06D0EA8
:10097000E66E740E0DEC0AF00101E55106E160EC43
:100980000AF0E66E17EC37F005D060EC0AF0E66E80
:1009900050EC37F045E946E9E7CFD9FF1200D9CF4F
:1009A000E6FFE1CFD9FF81E958E8136A146A156AB6
:1009B000166A176A186AE70E926ED00E936EB80E1A
:1009C000946EF19E8A86D0B604D0E66ABAEC2FF017
:1009D00041E9170EE66E55EC3EF041E959EC0AF09C
:1009E000750EE66E1AEC3EF041E990EC0AF001015A
:1009F000E451FF0A02E175EF09F0F40A01E16AD35C
:100A0000010A01E1C4D2030A01E12DD2010A01E188
:100A100017D20F0A01E1FED1010A01E1D5D1030A83
:100A200001E1BFD1010A01E1AAD1070A01E1A2D186
:100A3000010A01E196D1030A01E187D1010A02E02E
:100A400083EF09F0760EF66E780EF76E0900F5CF9B
:100A500060F00900F5CF61F00900F5CF62F0090000
:100A6000F5CF63F00900F5CF64F00900F5CF65F02C
:100A70000900F5CF66F00900F5CF67F00900F5CF62
:100A800068F00900F5CF69F00900F5CF6AF00900B8
:100A9000F5CF6BF00900F5CF6CF00900F5CF6DF0E4
:100AA0000900F5CF6EF00900F5CF6FF00900F5CF22
:100AB00070F00900F5CF71F00900F5CF72F0090070
:100AC000F5CF73F00900F5CF74F00900F5CF75F09C
:100AD0000900F5CF76F00900F5CF77F00900F5CFE2
:100AE00078F00900F5CF79F00900F5CF7AF0090028
:100AF000F5CF7BF00900F5CF7CF00900F5CF7DF054
:100B00000900F5CF7EF00900F5CF7FF00900F5CFA1
:100B100080F00900F5CF81F00900F5CF82F00900DF
:100B2000F5CF83F00900F5CF84F00900F5CF85F00B
:100B30000900F5CF86F00900F5CF87F00900F5CF61
:100B400088F00900F5CF89F00900F5CF8AF0090097
:100B5000F5CF8BF00900F5CF8CF00900F5CF8DF0C3
:100B60000900F5CF8EF00900F5CF8FF00900F5CF21
:100B700090F00900F5CF91F00900F5CF92F009004F
:100B8000F5CF93F00900F5CF94F00900F5CF95F07B
:100B90000900F5CF96F00900F5CF97F00900F5CFE1
:100BA00098F00900F5CF99F00900F5CF9AF0090007
:100BB000F5CF9BF00900F5CF9CF00900F5CF9DF033
:100BC0000900F5CF9EF00900F5CF9FF00900F5CFA1
:100BD000A0F00900F5CFA1F00900F5CFA2F00900BF
:100BE000F5CFA3F00900F5CFA4F00900F5CFA5F0EB
:100BF0000900F5CFA6F00900F5CFA7F00900F5CF61
:100C0000A8F00900F5CFA9F00900F5CFAAF0090076
:100C1000F5CFABF00900F5CFACF00900F5CFADF0A2
:100C20000900F5CFAEF00900F5CFAFF00900F5CF20
:100C3000B0F00900F5CFB1F00900F5CFB2F009002E
:100C4000F5CFB3F00900F5CFB4F00900F5CFB5F05A
:100C50000900F5CFB6F00900F5CFB7F00900F5CFE0
:100C6000B8F00900F5CFB9F00900F5CFBAF00900E6
:100C7000F5CFBBF00900F5CFBCF00900F5CFBDF012
:100C80000900F5CFBEF00900F5CFBFF00900F5CFA0
:100C9000C0F00900F5CFC1F00900F5CFC2F009009E
:100CA000F5CFC3F00900F5CFC4F00900F5CFC5F0CA
:100CB0000900F5CFC6F00800F5CFC7F00001C7B7AF
:100CC0001CD02F0EC16F400EC06FC26FC787C79177
:100CD000C783C7953C0EC36FC46B0F0EC56FC66B41
:100CE000C789C78DC79BC78F600EE66E000EE66E84
:100CF000C4EC24F042E9680EC6DBF3EC20F097EC7C
:100D00002EF0D1EC27F0F4EC11F0E3EC1CF0DD0E4A
:100D1000F66E780EF76E0800F550080B02E1A7ECAE
:100D20002EF046EC2FF0380E946E82EC22F081A863
:100D300084D00001C7A907D00101010EE46F0001B2
:100D4000C96BCA6BE0D2D4DBDED20001C8B303D0DA
:100D50000101020EE46F020E0101E55D01E0D3D254
:100D600031D00001C8B3C4DB020E0101E55D01E032
:100D7000CAD228D0C5DBC8A1C6D2010123D0E8DB86
:100D8000CCBFCD69BAEC0AF0A5DB0001C8A102D046
:100D90000101E4690101CB5101E1B5D20101050E68
:100DA000B1D2C0C0C9F0C1C0CAF0630EE66E740E05
:100DB00034DB0101CB5102E10101A2DB0001C8A13A
:100DC000A2D20101E4699FD2E551020A15E0030AAB
:100DD00007E0010A1BE1BCDBCCBFCD69CBDB0AD04D
:100DE0005E0EE66E740E19DBECEC2EF0F3CFE6FF30
:100DF000F4CFE6FF6FDB0AD0E56B0001C8A306D095
:100E0000C9693F0ECA6F0101010EE86F0001C8B346
:100E10007AD276D2E551020A06E0020A02E0010A1D
:100E200003E12ADD01D0E56B0001C8A303D0010175
:100E3000080EE46F0001C8B166D20101030E62D250
:100E40007D0EE66EFAEC3DF041E9000EE66EE66AD4
:100E5000A4EC3EF042E90101E56B2BDB156A166A52
:100E60000101090EE46F63DB000A1EE0010A18E0CD
:100E7000030A12E0010A0CE0070A06E0010A18E181
:100E8000590EE66E740E13D0540EE66E740E0FD02B
:100E90004F0EE66E740E0BD04A0EE66E740E07D03F
:100EA000450EE66E740E03D0400EE66E740EB5DA93
:100EB0000001C8B302D00101E469BCEC3EF011DBD3
:100EC00001E321D2BCEC3EF0ECDAA4EC3EF042E9C6
:100ED000152A000E1622020EE66EE66AC5C0E6FF6F
:100EE000C6C0E6FF92EC2DF0FE0EE350155C41E922
:100EF000E550165801E207D200C2DAF001C2DBF079
:100F000002C2DCF003C2DDF004C2DEF005C2DFF095
:100F100006C2E0F007C2E1F00101E56B01010351F7
:100F2000056E0451066E0551076E0651086E075195
:100F3000096E08510A6E09510B6E0A510C6E0B5165
:100F40000D6E0C510E6E0D510F6E0E51106EE66A45
:100F5000C7EC28F041E9116A126AD890125004E6F1
:100F60005E0E115C010E125802E272DAF6D7C9C0A9
:100F7000E6FFC7EC28F041E9BDEC3FF001010A0EA5
:100F8000E46F02014651176E4751186EBCD1E5510E
:100F9000030A31E0010A06E0020A02E0010A2CE13C
:100FA0006BDC2AD0C4DA000A14E01750E708030EFD
:100FB000185412E23B0EE66E740E2FDA0101E80EB1
:100FC000175CCC6F030E1858CD6FCCC1E6FFE66EF0
:100FD0000BD00101E56B10D0360EE66E740E1DDAF3
:100FE00017EBE6FF18EBE6FF030EE66ECF0EE66E9C
:100FF000000EC5DA01D0E56B020E0001C8155DE1F7
:101000000101E7515AE193DA010A49E0030A3EE09F
:10101000010A38E0070A32E0010A45E1CB510C0D24
:1010200002018851F324E96E8951F420EA6E05EB40
:10103000EEFF06EBEEFF07EBEEFF08EBEEFF09EB32
:10104000EEFF0AEBEEFF0BEBEEFF0CEBEEFF0DEB12
:10105000EEFF0EEBEEFF0FEBEEFF10EBEEFF0001ED
:10106000CB2B380ECB5D1FE301010B0EE46F0001AB
:10107000CB6BCC6B98EC26F074DA15D0D8D943EC56
:101080001FF010D0D4D9FEEC1EF00CD0D950050FB3
:10109000E66EDACFE6FF58EC1FF042E904D0C7D97C
:1010A00063EC1EF048E90001C7AD04D00101010E58
:1010B000E76F03D00101070EE46F020E0001C815AF
:1010C00001E121D10101E75101E11DD1080EE46FD9
:1010D000E76B19D10001CC51010BE66EACEC26F0A8
:1010E00041E9C6D90001CC2B310EE66E740E95D9BC
:1010F0000001CC51E66EE66A020EE66ED00EE66E98
:10110000000E3DDA640E0001CC5D01E0FCD0A0C70A
:1011100060F0A1C761F0A2C762F0A3C763F0A4C7E3
:1011200064F0A5C765F0A6C766F0A7C767F0A8C7B3
:1011300068F0A9C769F0AAC76AF0ABC76BF0ACC783
:101140006CF0ADC76DF0AEC76EF0AFC76FF0B0C753
:1011500070F0B1C771F0B2C772F0B3C773F0B4C723
:1011600074F0B5C775F0B6C776F0B7C777F0B8C7F3
:1011700078F0B9C779F0BAC77AF0BBC77BF0BCC7C3
:101180007CF0BDC77DF0BEC77EF0BFC77FF0C0C793
:1011900080F0C1C781F0C2C782F0C3C783F0C4C763
:1011A00084F0C5C785F0C6C786F0C7C787F0C8C733
:1011B00088F0C9C789F0CAC78AF0CBC78BF0CCC703
:1011C0008CF0CDC78DF0CEC78EF0CFC78FF0D0C7D3
:1011D00090F0D1C791F0D2C792F0D3C793F0D4C7A3
:1011E00094F0D5C795F0D6C796F0D7C797F0D8C773
:1011F00098F0D9C799F0DAC79AF0DBC79BF0DCC743
:101200009CF0DDC79DF0DEC79EF0DFC79FF0E0C712
:10121000A0F0E1C7A1F0E2C7A2F0E3C7A3F0E4C7E2
:10122000A4F0E5C7A5F0E6C7A6F0E7C7A7F0E8C7B2
:10123000A8F0E9C7A9F0EAC7AAF0EBC7ABF0ECC782
:10124000ACF0EDC7ADF0EEC7AEF0EFC7AFF0F0C752
:10125000B0F0F1C7B1F0F2C7B2F0F3C7B3F0F4C722
:10126000B4F0F5C7B5F0F6C7B6F0F7C7B7F0F8C7F2
:10127000B8F0F9C7B9F0FAC7BAF0FBC7BBF0FCC7C2
:10128000BCF0FDC7BDF0FEC7BEF0FFC7BFF0CD513B
:10129000070BF36EF80EC715F310C76F600EF3D887
:1012A000116A126A640ED89012BE03D0115C000E4F
:1012B000125802E2CDD8F6D72BD9640ED89012BEC0
:1012C00003D0115C000E125802E2C2D8F6D720D922
:1012D000640ED89012BE03D0115C000E125802E2C8
:1012E000B7D8F6D701010A0E0DD0E8C1E6FFBAEC77
:1012F0002FF041E91CD9CD6FC781C793C785CB6B50
:101300000101070EE46FC7EC15F00001C86B8150B6
:10131000100B01E0010EC8273EEC2FF0000906E09B
:10132000020E0001C827FCD8136A146AC7EC15F036
:101330003AEC04F08DEC22F0C7EC15F0040E01013C
:10134000E76E661902E7663502D06651E75C12E285
:101350002C0EE66E740E61D8E66A650EE66E010E1E
:10136000E66E010EE66ED00EE66E000EE66E75ECD1
:1013700037F046E9CE0EE66E000EE66E2EEC29F052
:1013800042E91CEC3FF000D90001C2510101CF6BD2
:10139000C2C0CFF1CE6BF350CE5DF450CF590CE20A
:1013A0000101E52B0A0EE45D04E141D8B4EC28F01C
:1013B00048E946EC2FF07DD8C7EC15F0ECEC3EF098
:1013C00090D822E2ECEC3EF06CD8D4EC3EF042E94E
:1013D000132A000E14220001C351C41115E0140E8B
:1013E000E66EE66AC3C0E6FFC4C0E6FF92EC2DF0ED
:1013F000FE0EE350D8801354145041E9E55804E23E
:10140000E66ABAEC2FF041E9C7EC15F0C9C0E6FF77
:10141000C7EC28F041E9F7EF04F0E66EE66ACE0E7D
:10142000E66E000EE66E47EC35F045E91200DEC0D0
:10143000E6FFDFC0E6FFE0C0E6FFE1C0E6FFDAC09E
:10144000E6FFDBC0E6FFDCC0E6FFDDC0E6FF120022
:101450008A84990EE66E85EC3FF041E98A94990EF4
:10146000E66E85EC3FF041E9112A000E12221200CF
:1014700078D80101CC51016ECD51026ECE51036E70
:10148000CF51046E1200E66EE66A600EE66E000E44
:10149000E66E760EE66E780EE66EA5EC1DF046E979
:1014A000120072D80101A80ECC5F610ECD5BBAEFBD
:1014B0000AF0000EE66EE66A04EC3FF042E9120024
:1014C00003EBE6FF04EBE6FF05EBE6FFCE0EE66E70
:1014D000000E1200030EE66ECE0EE66E000EBFEF9B
:1014E0000AF052D80101F350A808610EF45412001A
:1014F0000101060EE46FC0C0C9F0C1C0CAF01200FD
:10150000040EE46F0001010EC96F110ECA6F1200C4
:101510001E0EE66E3AEC3EF041E9116A126A1200C4
:10152000000EE66EE66AD4EC3EF042E912000001DD
:10153000C751070B120001EBE6FF02EBE6FF03EBDE
:10154000E6FF04EBE6FFC7EC35F048E938EF0AF0B8
:10155000680EE66E740E61DFA1C2CCF10101CD6BA5
:101560001200A2C2CCF1A3C2CDF1A4C2CEF1A5C299
:10157000CFF11200CCC1E6FFCDC1E6FF1200E66E4E
:1015800017EC37F045E91200F3CFCCF1F4CFCDF1F1
:02159000120047
:0E15920003EBE6FF04EBE6FF05EBE6FF06EBDE
:1015A000E6FFEECFE6FFEECFE6FFEECFE6FFEECFB3
:1015B000E6FFD3EC35F007EBE6FF08EBE6FF09EBBF
:1015C000E6FF0AEBE6FF08E8EECFE6FFEECFE6FF28
:1015D000EECFE6FFEECFE6FFD3EC35F02D50292617
:1015E0002E502A222F502B2230502C2244E90BEB74
:1015F000E6FF0CEBE6FF0DEBE6FF0EEBE6FF08E87F
:10160000EECFE6FFEECFE6FFEECFE6FFEECFE6FF52
:10161000D3EC35F02D5029262E502A222F502B2284
:1016200030502C2244E908E8EECFE6FFEECFE6FF8B
:10163000EECFE6FFEECFE6FF2D5029262E502A22D0
:101640002F502B2230502C2244E924E903EBE6FFF3
:1016500004EBE6FF05EBE6FF06EBE6FFEECFE6FF69
:10166000EECFE6FFEECFE6FFEECFE6FFD3EC35F0B0
:1016700007EBE6FF08EBE6FF09EBE6FF0AEBE6FF08
:1016800008E8EECFE6FFEECFE6FFEECFE6FFEECFC7
:10169000E6FFD3EC35F031502D2632502E22335058
:1016A0002F223450302244E90BEBE6FF0CEBE6FF2F
:1016B0000DEBE6FF0EEBE6FF08E8EECFE6FFEECF20
:1016C000E6FFEECFE6FFEECFE6FFD3EC35F031508C
:1016D0002D2632502E2233502F223450302244E90E
:1016E00008E8EECFE6FFEECFE6FFEECFE6FFEECF67
:1016F000E6FF31502D2632502E2233502F22345007
:10170000302244E924E903EBE6FF04EBE6FF05EBB6
:10171000E6FF06EBE6FFEECFE6FFEECFE6FFEECF0D
:10172000E6FFEECFE6FFD3EC35F007EBE6FF08EB84
:10173000E6FF09EBE6FF0AEBE6FF08E8EECFE6FF7F
:10174000EECFE6FFEECFE6FFEECFE6FFD3EC35F0CF
:101750003550312636503222375033223850342219
:1017600044E90BEBE6FF0CEBE6FF0DEBE6FF0EEBBF
:10177000E6FF08E8EECFE6FFEECFE6FFEECFE6FFAE
:10178000EECFE6FFD3EC35F035503126365032221D
:10179000375033223850342244E908E8EECFE6FFD0
:1017A000EECFE6FFEECFE6FFEECFE6FF3550312677
:1017B00036503222375033223850342244E924E95B
:1017C000E552E5500E6EE5500D6EE5500C6EE7509B
:1017D0000B6EE552E5500A6EE550096EE550086E55
:1017E000E750076EE552E550066EE550056EE55090
:1017F000046EE750036E000CD89006BED880063207
:1018000005320432D8900ABED8800A320932083232
:10181000D8900EBED8800E320D320C32000C036A06
:10182000046AEE50056EEE50066E076A086AEE50C6
:10183000096EEE500A6E0B6A0C6AEE500D6EEE5099
:101840000E6E000C64E8D9CFE6FFDACFE6FFE1CFF9
:10185000D9FFE2CFDAFFA9E901EBE9FF02EBEAFFEA
:1018600006E8DDDFC9DFC8DF00EE60F092DE83EB63
:101870000FF084EB10F085EB11F086EB12F087EBA4
:1018800013F088EB14F089EB15F08AEB16F08BEB74
:1018900017F08CEB18F08DEB19F08EEB1AF001EBD2
:1018A000E9FF02EBEAFFBBDFA7DFA6DFA5DF00EE63
:1018B00090F06FDE03EBE6FF04EBE6FF05EBE6FFDF
:1018C00006EBE6FF03EBE6FF04EBE6FF05EBE6FFC6
:1018D00006EBE6FFD3EC35F007EBE6FF08EBE6FF9F
:1018E00009EBE6FF0AEBE6FF07EBE6FF08EBE6FF96
:1018F00009EBE6FF0AEBE6FFD3EC35F00BEBE6FF76
:101900000CEBE6FF0DEBE6FF0EEBE6FF0BEBE6FF65
:101910000CEBE6FF0DEBE6FF0EEBE6FFD3EC35F04C
:1019200031502D2632502E2233502F223450302267
:1019300044E92D5029262E502A222F502B22305098
:101940002C2244E90201295038272A5039232B50F0
:101950003A232C503B23FC0EE3CFE6FFE3CFE6FF18
:10196000E3CFE6FFE3CFE6FF7EEC36F0FC0EE3CFFD
:10197000E6FFE3CFE6FFE3CFE6FFE3CFE6FF03EBCF
:10198000E6FF04EBE6FF05EBE6FF06EBE6FFD3EC34
:1019900035F0E552E550066EE550056EE550046EF3
:1019A000E750036EFC0EE3CFE6FFE3CFE6FFE3CFA5
:1019B000E6FFE3CFE6FF07EBE6FF08EBE6FF09EB08
:1019C000E6FF0AEBE6FFD3EC35F0E552E5500A6E90
:1019D000E550096EE550086EE750076EFC0EE3CF48
:1019E000E6FFE3CFE6FFE3CFE6FFE3CFE6FF0BEB57
:1019F000E6FF0CEBE6FF0DEBE6FF0EEBE6FFD3ECAC
:101A000035F0E552E5500E6EE5500D6EE5500C6E6A
:101A1000E7500B6ED3EC35F00201295020272A50F5
:101A200021232B5022232C50232344E90FEBE6FFE4
:101A300010EBE6FF11EBE6FF12EBE6FF0FEBE6FF24
:101A400010EBE6FF11EBE6FF12EBE6FFD3EC35F00F
:101A500013EBE6FF14EBE6FF15EBE6FF16EBE6FFF4
:101A600013EBE6FF14EBE6FF15EBE6FF16EBE6FFE4
:101A7000D3EC35F017EBE6FF18EBE6FF19EBE6FFCA
:101A80001AEBE6FF17EBE6FF18EBE6FF19EBE6FFB4
:101A90001AEBE6FFD3EC35F031502D2632502E22D2
:101AA00033502F223450302244E92D5029262E5015
:101AB0002A222F502B2230502C2244E90201295097
:101AC0003C272A503D232B503E232C503F23FC0E15
:101AD000E3CFE6FFE3CFE6FFE3CFE6FFE3CFE6FFAA
:101AE0007EEC36F0FC0EE3CFE6FFE3CFE6FFE3CF7C
:101AF000E6FFE3CFE6FF0FEBE6FF10EBE6FF11EBAF
:101B0000E6FF12EBE6FFD3EC35F0E552E550126E3E
:101B1000E550116EE550106EE7500F6EFC0EE3CFEE
:101B2000E6FFE3CFE6FFE3CFE6FFE3CFE6FF13EB0D
:101B3000E6FF14EBE6FF15EBE6FF16EBE6FFD3EC52
:101B400035F0E552E550166EE550156EE550146E11
:101B5000E750136EFC0EE3CFE6FFE3CFE6FFE3CFE3
:101B6000E6FFE3CFE6FF17EBE6FF18EBE6FF19EB26
:101B7000E6FF1AEBE6FFD3EC35F0E552E5501A6EBE
:101B8000E550196EE550186EE750176ED3EC35F03E
:101B90000201295024272A5025232B5026232C507C
:101BA000272344E907EBE6FF08EBE6FF09EBE6FF36
:101BB0000AEBE6FF17EBE6FF18EBE6FF19EBE6FF93
:101BC0001AEBE6FFD3EC35F00BEBE6FF0CEBE6FF90
:101BD0000DEBE6FF0EEBE6FF13EBE6FF14EBE6FF83
:101BE00015EBE6FF16EBE6FFD3EC35F02D50295E42
:101BF0002E502A5A2F502B5A30502C5A44E90BEBB6
:101C0000E6FF0CEBE6FF0DEBE6FF0EEBE6FF0FEB5E
:101C1000E6FF10EBE6FF11EBE6FF12EBE6FFD3EC7D
:101C200035F003EBE6FF04EBE6FF05EBE6FF06EB22
:101C3000E6FF17EBE6FF18EBE6FF19EBE6FF1AEB02
:101C4000E6FFD3EC35F031502D5E32502E5A335032
:101C50002F5A3450305A44E903EBE6FF04EBE6FF19
:101C600005EBE6FF06EBE6FF13EBE6FF14EBE6FF02
:101C700015EBE6FF16EBE6FFD3EC35F007EBE6FFDE
:101C800008EBE6FF09EBE6FF0AEBE6FF0FEBE6FFEA
:101C900010EBE6FF11EBE6FF12EBE6FFD3EC35F0BD
:101CA0003550315E3650325A3750335A3850345AE4
:101CB00044E9E552E5501A6EE550196EE550186E8C
:101CC000E750176EE552E550166EE550156EE5507B
:101CD000146EE750136EE552E550126EE550116E2A
:101CE000E550106EE7500F6E0FEBE6FF10EBE6FFCE
:101CF00011EBE6FF12EBE6FF0FEBE6FF10EBE6FF62
:101D000011EBE6FF12EBE6FFD3EC35F013EBE6FF49
:101D100014EBE6FF15EBE6FF16EBE6FF13EBE6FF31
:101D200014EBE6FF15EBE6FF16EBE6FFD3EC35F020
:101D300017EBE6FF18EBE6FF19EBE6FF1AEBE6FF01
:101D400017EBE6FF18EBE6FF19EBE6FF1AEBE6FFF1
:101D5000D3EC35F031502D2632502E2233502F2225
:101D60003450302244E92D5029262E502A222F505B
:101D70002B2230502C2244E90201295040272A50BE
:101D800041232B5042232C504323FC0EE3CFE6FF8C
:101D9000E3CFE6FFE3CFE6FFE3CFE6FF7EEC36F0EE
:101DA000FC0EE3CFE6FFE3CFE6FFE3CFE6FFE3CFB2
:101DB000E6FF0FEBE6FF10EBE6FF11EBE6FF12EBA1
:101DC000E6FFD3EC35F0E552E550126EE550116EAA
:101DD000E550106EE7500F6EFC0EE3CFE6FFE3CF49
:101DE000E6FFE3CFE6FFE3CFE6FF13EBE6FF14EBFE
:101DF000E6FF15EBE6FF16EBE6FFD3EC35F0E55218
:101E0000E550166EE550156EE550146EE750136EF2
:101E1000FC0EE3CFE6FFE3CFE6FFE3CFE6FFE3CF41
:101E2000E6FF17EBE6FF18EBE6FF19EBE6FF1AEB10
:101E3000E6FFD3EC35F0E552E5501A6EE550196E29
:101E4000E550186EE750176ED3EC35F002012950BB
:101E500028272A5029232B502A232C502B2344E9AE
:101E6000100E0060B4D113EBE6FF14EBE6FF15EBA8
:101E7000E6FF16EBE6FF0BEBE6FF0CEBE6FF0DEBE8
:101E8000E6FF0EEBE6FFD3EC35F017EBE6FF18EBC1
:101E9000E6FF19EBE6FF1AEBE6FF07EBE6FF08EBC0
:101EA000E6FF09EBE6FF0AEBE6FFD3EC35F02D5039
:101EB000295E2E502A5A2F502B5A30502C5A44E962
:101EC00017EBE6FF18EBE6FF19EBE6FF1AEBE6FF70
:101ED00003EBE6FF04EBE6FF05EBE6FF06EBE6FFB0
:101EE000D3EC35F00FEBE6FF10EBE6FF11EBE6FF6E
:101EF00012EBE6FF0BEBE6FF0CEBE6FF0DEBE6FF6C
:101F00000EEBE6FFD3EC35F031502D5E32502E5AF9
:101F100033502F5A3450305A44E90FEBE6FF10EBA0
:101F2000E6FF11EBE6FF12EBE6FF07EBE6FF08EB3F
:101F3000E6FF09EBE6FF0AEBE6FFD3EC35F013EB27
:101F4000E6FF14EBE6FF15EBE6FF16EBE6FF03EB0F
:101F5000E6FF04EBE6FF05EBE6FF06EBE6FFD3EC5E
:101F600035F03550315E3650325A3750335A38508A
:101F7000345A44E9E552E550266EE550256EE550A9
:101F8000246EE750236EE552E550226EE550216E37
:101F9000E550206EE7501F6EE552E5501E6EE5508D
:101FA0001D6EE5501C6EE7501B6E1BEBE6FF1CEB35
:101FB000E6FF1DEBE6FF1EEBE6FF1BEBE6FF1CEB6F
:101FC000E6FF1DEBE6FF1EEBE6FFD3EC35F01FEB63
:101FD000E6FF20EBE6FF21EBE6FF22EBE6FF1FEB3F
:101FE000E6FF20EBE6FF21EBE6FF22EBE6FFD3EC7A
:101FF00035F023EBE6FF24EBE6FF25EBE6FF26EBCF
:10200000E6FF23EBE6FF24EBE6FF25EBE6FF26EBFE
:10201000E6FFD3EC35F031502D2632502E223350CE
:102020002F223450302244E92D5029262E502A22C6
:102030002F502B2230502C2244E97EEC36F0FC0E3F
:10204000E3CFE6FFE3CFE6FFE3CFE6FFE3CFE6FF34
:102050001BEBE6FF1CEBE6FF1DEBE6FF1EEBE6FFCE
:10206000D3EC35F0E552E5501E6EE5501D6EE5509F
:102070001C6EE7501B6EFC0EE3CFE6FFE3CFE6FFDE
:10208000E3CFE6FFE3CFE6FF1FEBE6FF20EBE6FF43
:1020900021EBE6FF22EBE6FFD3EC35F0E552E5500D
:1020A000226EE550216EE550206EE7501F6EFC0E4B
:1020B000E3CFE6FFE3CFE6FFE3CFE6FFE3CFE6FFC4
:1020C00023EBE6FF24EBE6FF25EBE6FF26EBE6FF3E
:1020D000D3EC35F0E552E550266EE550256EE5501F
:1020E000246EE750236E44E91BEBE6FF1CEBE6FF92
:1020F0001DEBE6FF1EEBE6FF1BEBE6FF1CEBE6FF2E
:102100001DEBE6FF1EEBE6FF02012D5014272E50BB
:1021100015232F50162330501723D3EC35F02950B8
:102120002C272A502D232B502E232C502F2344E9CB
:102130000FEBE6FF10EBE6FF11EBE6FF12EBE6FF1D
:102140000FEBE6FF10EBE6FF11EBE6FF12EBE6FF0D
:102150002D5018272E5019232F501A2330501B238F
:10216000D3EC35F0295030272A5031232B5032231D
:102170002C50332344E903EBE6FF04EBE6FF05EBC9
:10218000E6FF06EBE6FF03EBE6FF04EBE6FF05EBFD
:10219000E6FF06EBE6FF2D501C272E501D232F5087
:1021A0001E2330501F23D3EC35F0295034272A50FA
:1021B00035232B5036232C50372344E9020107EBFB
:1021C00008F208EB09F209EB0AF20AEB0BF2E5520E
:0E21D000E5CFDAFFE7CFD9FF64E9000C000C81
:0221DE00F3EC20
:1021E00016F031E021EC16F0D00F056E055009080D
:1021F00002E2070E055E05500F0802E2200E055EA2
:1022000005500F0815E30228E96E000E0320EA6E60
:10221000EF50D00F066E0650090802E2070E065E68
:1022200006500F0802E2200E065E06500F0802E27A
:10223000FF0E0AD00538F00B0624E66E3FEC16F0D0
:10224000E552E750EF6E000E89EF16F0F3EC16F052
:1022500024E044EC16F0C3DF44E900090BE1D95057
:10226000060FE4EC16F0020E4CEC16F0B8DF44E971
:10227000000902E0FF0E12D005500101CF6BCF6FB5
:10228000CE6B0650CE25CC6F000ECF21CD6F3FEC2C
:1022900016F0CCC1EEFFCDC1EDFF000E89EF16F0B8
:1022A0002EEC16F085E944E821EC16F048E044EC09
:1022B00016F0CCDF44E900090BE1D950070FE4EC3C
:1022C00016F0040E4CEC16F0C1DF44E9000902E000
:1022D000FF0E36D0E66A010EE66EE66AE66AE66A48
:1022E000E66EE66AE66A05EBE6FF06EBE6FFE66AFF
:1022F000E66AC6EC2DF0C6EC2DF0E552E5CFCFF145
:10230000E5CFCEF1E5CFCDF1E7CFCCF107EBD0F1C2
:1023100008EBD1F10101D26BD36BD051CC27D15155
:10232000CD23D251CE23D351CF233FEC16F0CCC1D5
:10233000EEFFCDC1EEFFCEC1EEFFCFC1EEFF000E2E
:1023400045E9E7CFD9FF12002EEC16F085E921EC24
:1023500016F010E021EC16F0300804E13FEC16F026
:10236000EF6A08D021EC16F0310806E13FEC16F0D8
:10237000010EEF6E000E01D0FF0E41E9E7CFD9FF4D
:1023800012002EEC16F081E942E8670E016E010E94
:10239000026E82EC16F00101CF6BCEBFCF69CEC1C9
:1023A000E6FFCFC1E6FF6FEC3CF056EC16F004E020
:1023B000012A000E0222EDD782EC16F0CF6BCEBFC1
:1023C000CF69CEC1E6FFCFC1E6FF8DEC3CF056EC05
:1023D00016F004E0012A000E0222EED701EBF3FF13
:1023E00002EBF4FF89EF16F0140E6F6E0201A66B7C
:1023F0000201A76B0201A86B33EC16F0DBEC16F0C0
:102400000101876BC86BCB6BC96BCA6B12001F0EC7
:102410000101D8808755E66E87C1CCF10101CD6BF3
:10242000CCBFCD69670ECC27010EE8EC16F060EC4E
:1024300032F043E912000001E35106E1DBDB91ECED
:1024400032F042E90201B46B1200FF0012002EECE0
:1024500016F081E963E80168DBEC16F001016751D1
:10246000510A01E1F8D1010A01E1E8D1020A01E1D2
:1024700088D1010A01E153D1100A01E132D1040AE5
:1024800001E1D7D0110A0EE01E0A01E02AD3016A49
:10249000270EE66E740EFDEC16F045E90101010E03
:1024A000CB6F1FD36851520A01E1B3D01F0A01E17B
:1024B0008ED00F0A01E17AD00A0A6DE00E0A60E0C0
:1024C000090A53E01C0A42E0030A31E0040A26E04C
:1024D000100A13E0080A01E004D3C00EE66E000EF5
:1024E0009DDBC00EE66E000EE66E010EC8EC16F027
:1024F000C0C0E6FFC7EC28F00FD0C10EE66E000E9C
:102500008DDBC10EE66E000EE66E010EC8EC16F015
:10251000C1C0E6FFAFEC29F041E9E3D2C20EE66E9E
:10252000000E7CDBC20EE66E000EE66E70D0B4ECE0
:1025300016F001E1051C04E004EBC3F005EBC4F068
:10254000010EE66EC30EE66E000E70D0B4EC16F00F
:1025500001E1051C04E004EBC5F005EBC6F0010E3B
:10256000E66EC50EE66E000E61D0E7DB05E00250B8
:102570000001C799E8B0C7890001C7B921D023D0AD
:10258000DCDB05E002500001C79BE8B0C78B00010F
:10259000C7AB19D015D0D1DB05E002500001C79DB3
:1025A000E8B0C78D0001C7AD0ED00AD0C6DB05E08C
:1025B00002500001C79FE8B0C78F0001C7AF03D02A
:1025C0000101310E02D00101300E886F8AD20268FB
:1025D000D950020F0CDB03DE44E9016EFF0E025CF2
:1025E0000BE002500001070BF36EF80EC715F31055
:1025F000C76F0101010EC86F0001C751070B026EC2
:10260000010EE66ED950020FE66EDACFE6FF010E3C
:10261000B6D0AADB01E1051C04E004EB46F205EBB1
:1026200047F2010EE66E460EE66E020EE66E020EF2
:10263000A6D0016A6851580A4FE00A0A3AE0040A33
:102640002DE01F0A27E01D0A21E0170A1BE00E0AF1
:102650000EE00A0A01E07AD060DB030E025C01E3BF
:1026600040D2E66A0101D9500C0FC9DAF6D755DB22
:10267000030E025C01E335D2E66A0101D950180F5E
:10268000BEDAF6D7B7DA29EC2FF00BD0B3DAECECE0
:102690002EF007D0AFDA01EC2FF003D0ABDA19EC53
:1026A0002FF0F3CFE6FFF4CFE6FFCDEC38F044E9AE
:1026B00018D294DB47EC35F045E902C2E6FF03C2CD
:1026C000E6FF030E9DDB17EC37F045E906C2E6FF97
:1026D00007C2E6FF020EA9D0FF0EE66E730E8DDB79
:1026E000ABD0016A680EE66EE66A600EE66E000E1A
:1026F000E66E760EE66E780EE66EA5EC1DF046E907
:102700000101C85104E0FAEC1CF00101C86BC95189
:10271000CA1101E1E6D1020EC96FCA6BE2D1300ED7
:10272000695D026E0250090802E2070E025E025065
:102730000F0802E2200E025E02500F0801E2D1D122
:10274000016A68514D0A0FE00A0A02E00168C9D126
:1027500024DB900E0101CC27000E69DA900E0101F6
:10276000CC27000E0AD019DB600E0101CC27000E29
:102770005EDA600E0101CC27000E2ADB040E08DBB6
:10278000B0D1D950040F33DA61DD44E9016E015054
:1027900001E0A7D10001C751070B010A3CE0010A83
:1027A0003AE0020A1BE0010A07E0070A01E099D1BA
:1027B0002DDA13EC1FF032D029DA13EC1FF046E9C2
:1027C000F50EE66E730E1FDB88DA040E19DB8ADA6B
:1027D000040EE66E8D0EE66E010E2BD009DB79DA63
:1027E00074DA78EC1FF046E9026A060E025C10E229
:1027F000090E0202F350036EE66A0101D9500C0F74
:10280000A2DA0350B8DA76DA200EEF6E022AEDD79C
:1028100071DAEF6A66D1FAD9B0EC1EF046E9DEDA79
:102820005CDA030EEDDA5EDA030EE66E8C0EE66E0F
:10283000010EE66E50EC37F045E953D1520E685D5B
:1028400001E04FD1470E695D01E04BD1010EC96F28
:10285000CA6B016A46D1760EF66E780EF76E0900E5
:10286000F5CF60F00900F5CF61F00900F5CF62F017
:102870000900F5CF63F00900F5CF64F00900F5CF4A
:1028800065F00900F5CF66F00900F5CF67F00900A3
:10289000F5CF68F00900F5CF69F00900F5CF6AF0CF
:1028A0000900F5CF6BF00900F5CF6CF00900F5CF0A
:1028B0006DF00900F5CF6EF00900F5CF6FF009005B
:1028C000F5CF70F00900F5CF71F00900F5CF72F087
:1028D0000900F5CF73F00900F5CF74F00900F5CFCA
:1028E00075F00900F5CF76F00900F5CF77F0090013
:1028F000F5CF78F00900F5CF79F00900F5CF7AF03F
:102900000900F5CF7BF00900F5CF7CF00900F5CF89
:102910007DF00900F5CF7EF00900F5CF7FF00900CA
:10292000F5CF80F00900F5CF81F00900F5CF82F0F6
:102930000900F5CF83F00900F5CF84F00900F5CF49
:1029400085F00900F5CF86F00900F5CF87F0090082
:10295000F5CF88F00900F5CF89F00900F5CF8AF0AE
:102960000900F5CF8BF00900F5CF8CF00900F5CF09
:102970008DF00900F5CF8EF00900F5CF8FF009003A
:10298000F5CF90F00900F5CF91F00900F5CF92F066
:102990000900F5CF93F00900F5CF94F00900F5CFC9
:1029A00095F00900F5CF96F00900F5CF97F00900F2
:1029B000F5CF98F00900F5CF99F00900F5CF9AF01E
:1029C0000900F5CF9BF00900F5CF9CF00900F5CF89
:1029D0009DF00900F5CF9EF00900F5CF9FF00900AA
:1029E000F5CFA0F00900F5CFA1F00900F5CFA2F0D6
:1029F0000900F5CFA3F00900F5CFA4F00900F5CF49
:102A0000A5F00900F5CFA6F00900F5CFA7F0090061
:102A1000F5CFA8F00900F5CFA9F00900F5CFAAF08D
:102A20000900F5CFABF00900F5CFACF00900F5CF08
:102A3000ADF00900F5CFAEF00900F5CFAFF0090019
:102A4000F5CFB0F00900F5CFB1F00900F5CFB2F045
:102A50000900F5CFB3F00900F5CFB4F00900F5CFC8
:102A6000B5F00900F5CFB6F00900F5CFB7F00900D1
:102A7000F5CFB8F00900F5CFB9F00900F5CFBAF0FD
:102A80000900F5CFBBF00900F5CFBCF00900F5CF88
:102A9000BDF00900F5CFBEF00900F5CFBFF0090089
:102AA000F5CFC0F00900F5CFC1F00900F5CFC2F0B5
:102AB0000900F5CFC3F00900F5CFC4F00900F5CF48
:102AC000C5F00900F5CFC6F00800F5CFC7F0C86B18
:102AD000CB6B010EC91904E1CA5102E1C96BCA6B83
:102AE000016A015064E9E7CFD9FF1200B7D881E944
:102AF00043E88DDC016E015042E00A0EE66E670E7F
:102B0000E66E010EE66E33EC35F043E9F350026EEB
:102B1000F450036E0150010187271F0EE76E8719DD
:102B200002E7E73402D0E750875D09E3010EF36E58
:102B3000F46AF3508708026E010EF454036E0250DB
:102B400003101DE002EBE9FF03EBEAFFEF6A7FDC15
:102B5000000906E0610EE66E7F0EE66E000E05D0FF
:102B60005C0EE66E7F0EE66E000E4AD917EC35F06D
:102B700045E90101876B77D80201010EB46F0201AC
:102B8000B45101E058DC44E9E7CFD9FF1200F6EC7C
:102B900037F018EC38F00201A651030827E2060EC0
:102BA000A65D24E3A3DFBCEC32F00101CA3508E2E4
:102BB000C9510108000ECA5503E2C92B000ECA23F1
:102BC0000A0EC91913E1CA5111E1E668E66AF9EC87
:102BD0001DF042E916EC38F00101C96BCA6BC90758
:102BE000000ECA5BC951CA11FAE12FDC1200ECD801
:102BF000D4EF16F0880EE66E010EE66E1200A3D832
:102C0000090E0202F350B7D8022A1200F1D8D950A7
:102C1000060FDAD8D950040FE4EF16F0E66EC4D8E8
:102C2000EFEC10F044E9016E010EE66E1200D0D810
:102C3000BBD850EC11F044E9016E010EE66ECDEF09
:102C400016F002EBE9FF03EBEAFFEF501200A4ECF1
:102C500011F044E9016EFF0E025C1200D9CFE6FFCD
:102C6000E1CFD9FF1200200EE66EE66AE66A670E33
:102C7000E66E010EE66ED9EC34F045E9120000EB89
:102C8000E9FF01EBEAFF1200D950050F9DD802EBD6
:102C9000E6FF03EBE6FF120001010224CC6F000EF9
:102CA0000320CD6FCCC1E6FFE66E120042E9F3CF00
:102CB000CCF1F4CFCDF10101F350F410120026EC69
:102CC00011F044E9016E041C1200D9500C0FE4EF1E
:102CD00016F0D950180FE4EF16F047EC35F045E93F
:102CE000F8EF16F017EC37F045E906EBE6FF07EBD7
:102CF000E6FF1200080E0324EA6A880FE96E010E4F
:102D0000EA22120001EBE9FF02EBEAFFEFCFCEF17E
:102D1000120043E9E7CFD9FF1200030EE66E010E61
:102D2000E66ED3DFD6DFFFEC1CF046E90C0EE66E54
:102D3000740E63D845E9026A12000268D950020F86
:102D400056DF27EF16F0CE6FDACFCFF10250040D29
:102D5000CE51F324CC6FDA50F420CD6FCCC1E6FF16
:102D6000E66E040EE66E120004680568D950040F82
:102D70003EDF5FEF16F0D16B880FD06F010ED123CD
:102D8000D0C1E6FFD1C1E6FF75EC37F046E912008D
:102D900037D875EC37F046E912000250040DF3CF36
:102DA000CCF1F4CFCDF11200C1EC11F0F3CFE6FF7E
:102DB000F4CFE6FF1200400EE66EE66AE66A1ADF1E
:102DC000D9EC34F045E91200E66EDACFE6FF1200E6
:102DD000CD23CCC1E6FFCDC1E6FF1200040EE66EA6
:102DE000740E03EF17F03ADF85E942E821EF16F0A1
:102DF00004EBE6FF05EBE6FF120005D847EF35F0E0
:0E2E0000E66EFAEF15F0E66EE66AFAEF15F0F0
:022E0E000000C2
:102E100000000000000000000000000000000000B2
:102E200000000000000000000000000000000000A2
:102E30000000000000000000000000000000000092
:102E40000000000000000000000000000000000082
:0639C00000000000000001
:0A39C6000201000E886F050E896FE4
:1039D000020EE66EF00EE66E460EE66E020EE66E25
:1039E00052D944E90201461D04E1471D02E1466B3C
:1039F000476B12000201466B476BE6EF1FF0EBDBF3
:103A000041E8076AD890075002E6030E075C45E2DA
:103A100000EBE9FF01EBEAFF6FDB0101D56BD4BFDF
:103A2000D569FFDACFAF02D0D069D1690D0E1F0B77
:103A300003E0010168DBFEE107EBCCF10101CD6B96
:103A4000CCBFCD6941DB0224E96ECD51032006DBFA
:103A500000EBE9FF01EBEAFF060EE926000EEA2281
:103A60004BDBD56BD4BFD569DCDACFAF02D0D069E0
:103A7000D1690E0E1F0B03E0010145DBFEE107EBF0
:103A8000CCF10101CD6BCCBFCD691EDB0424E96E06
:103A9000CD510520E3DA072AB5D742E9E7CFD9FFB0
:103AA0001200D9CFE6FFE1CFD9FF85E942E802EB6A
:103AB000F6FF03EBF7FFF86AA68EA69CA684A688FD
:103AC000F250800B01E0010E066EF29E550EA76EBD
:103AD000AA0EA76EA68200000650E8B0F28EE8A0FB
:103AE000F29EA694056A400E055C2BE20550002468
:103AF000E96E000E0120EA6EEF50F56E0D0005280C
:103B00001F0B1DE1200EF65E000EF75A000EF85A4C
:103B1000A68EA69CA684A698F250800B01E0010E0A
:103B2000066EF29E550EA76EAA0EA76EA682000024
:103B3000A694200EF626000EF722000EF822052A83
:103B4000D2D743E9E7CFD9FF120045DB7FE845E84C
:103B50003F0E0414076EC00E0414086EFF0E051409
:103B6000096E400EE66EE66A08EBE6FF09EBE6FF3B
:103B7000E66AD9500B0F24DBB6EC34F047E900506D
:103B8000011026E0D890075002E6400E075C20E2C4
:103B9000C1DAEF50E66E0101D9500B0FCC6FDACFCE
:103BA000CDF107EBCEF1CF6BCEBFCF69CC51CE2597
:103BB000E96ECD51CF21EA6EE552E750EF6E072A4C
:103BC000042A000E0522022A03220006015AD7D732
:103BD000D9500B0FF5DA08EBE6FF09EBE6FF61DFE2
:103BE00044E900500110B4E17FE946E9E7CFD9FF8D
:103BF0001200D9CFE6FFE1CFD9FF83E941E8A6A2C1
:103C000002D00000FCD700EBA9FF01EBA8FFA69EA5
:103C1000A69CA698A684F250800B01E0010E036ECC
:103C2000F29E550EA76EAA0EA76EA6820350E8B0AC
:103C3000F28EE8A0F29EA69442E9E7CFD9FF1200E7
:103C4000EBD984E900EBA9FFA69EA69CA68001EB18
:103C5000E9FF02EBEAFFA8CFEFFF61D2DDD985E9EA
:103C6000005010E003EBE6FF01EBE9FF02EBEAFF97
:103C7000EFCFE6FFBEDF42E90006012A000E022276
:103C8000032AEED74CD2C8D985E943E882EB05F088
:103C900083EB06F081EB07F0A6B2FED7A1980050A7
:103CA0000EE007EBE6FF05EBE6FF06EBE6FFC8DFFD
:103CB00043E90006052A000E0622072AF0D744E948
:103CC000E7CFD9FF1200A8D989E942E8020146519D
:103CD000DC08050E475502E2466B476BB50EE66EF3
:103CE000E66A06EBE6FF07EBE6FF92EC2DF0E55205
:103CF000E5500A6EE750096E5A0E01010224CC6F9E
:103D0000000E0320CD6FCC510926CD510A22020EA0
:103D1000E66ED950090F54DA020EE66EE66AA8D9AB
:103D20005DDAA6D909DA0101CC51CD1114E1400EBA
:103D3000E66EE66A16D9400ECC5F000ECD5B010E32
:103D400088D9FEE115DA200ECC5F000ECD5B010EA6
:103D500080D9FEE137D93AD943E9E7CFD9FF12003C
:103D60003ADA42E8C00E87D9C00EB6D910E1CF5179
:103D7000CD190DE102014651005C4751015807E29F
:103D8000020EE66EE66EE66A400E2BD90BD0CBD95A
:103D9000010ED890F636F736E806FBE109DA0A009C
:103DA000F550086EB50E71D9C7D901015A0ECC5F16
:103DB000000ECD5BAFD9CCC1EEFFCDC1EDFFB50E8E
:103DC000E66EE66A62D90101FE0EE350075CCE6F33
:103DD00041E9E5500858CF6FCEC1E6FFE66ED1EC61
:103DE0002CF0AAD904EBE9FF05EBEAFFCCC1EEFF0A
:103DF000CDC1EDFF43E9E7CFD9FF12000DD974D94A
:103E000002E2466B476B49D9FAD847D9BDD809E1D8
:103E1000C8D91FD9FEE1ACD9100E51D91AD9FEE18B
:103E2000D1D8D4D885D1D7D944E8E00E24D9E00E32
:103E300053D910E1CF51CD190DE102014651005C7B
:103E40004751015807E2040EE66EE66EE66A200E60
:103E5000C8D80BD068D9020ED890F636F736E806E7
:103E6000FBE1EFD80800F5500A6E54D909EBEEFFDC
:103E70000AEBEDFF04EBE9FF05EBEAFF07EBEEFFD2
:103E800008EBEDFF55D1C8D82FD902E2466B476B3E
:103E90000DD9B5D80BD978D809E183D9DAD8FEE1A4
:103EA00067D9100E0CD9D5D8FEE18CD88FD840D167
:103EB000B3D883E90C0E88D946C2CCF147C2CDF104
:103EC0000101CD03F3CFCDF1CC03F3CFCCF1F4500E
:103ED000CD270E0E53D90201462B000E4723FA0EB2
:103EE000465D000E475902E3466B476B6FD817D10A
:103EF00072D94CE818D90C0EF702F3CFF7FFF6028F
:103F0000F3CFF6FFF450F7269CD80900F5500A6E5F
:103F10000900F5500B6E0900F5500C6E0900F550C4
:103F20000D6E0900F5500E6E0900F5500F6E090078
:103F3000F550106E0900F550116E0900F550126E23
:103F4000D950070F3DD904EBE6FF05EBE6FF02EB86
:103F5000E6FF03EBE6FF53DD46E94DE9E7CFD9FF86
:103F60001200480EE66E020EE66E8DDE44E9400E4B
:103F7000E66EE66A480EE66E020EE66E46C2CCF1CA
:103F800047C2CDF10101120000EBE6FF01EBE6FFB5
:103F900002EBE6FF03EBE6FFDDD80B6ECF510C6EB4
:103FA000040EE66ED950090F0BD9040EE66EE66AD0
:103FB000200EC8D813D9200EC5D8BED80101CC51C7
:103FC000CD1112000E0E0101BEEF20F0020EE66EC2
:103FD000460EE66E020EE66EF00EE66E3FDE44E939
:103FE0001200F2D8D4EC2CF092EC2DF0A5D8CCC174
:103FF000E6FFD950070FE4D846DE44E9120004EB8F
:10400000E6FF05EBE6FF06EBE6FF07EBE6FFA2D8CF
:10401000096ECF510A6E1200D9CFE6FFE1CFD9FF6A
:104020001200D890D437D537D251D425E96ED35168
:10403000D521EA6EEECFCEF1EFCFCFF1D06BD16BC1
:104040001200B6D80900F550086E0900F550096E47
:104050001200D890CC37CD37E8061200EA6ECEC1F8
:10406000EEFFCFC1EEFFD0C1EEFFD1C1EEFF1200D7
:10407000400EA2EF20F0020146150101CC6FFF0EA9
:10408000020147150101CD6F1200E66EE66A07EBEB
:10409000E6FF08EBE6FFD4EF2CF0E0C1E6FFE1C15C
:1040A000E6FFE2C1E6FFE3C1E6FF1200DCC1E6FF86
:1040B000DDC1E6FFDEC1E6FFDFC1E6FF1200CC5F37
:1040C000000ECD5B020E1200D890CC37CD37D890C1
:1040D000CC37CD37CC5112000014CE6FFF0E011437
:1040E000CF6FCE51CC19120089E944E80201465144
:1040F000EE08020E47551200E9CFD2F1EACFD3F114
:1041000007EBD4F11200D890CE37CF37D037D13764
:10411000E806120002EBE9FF03EBEAFF120041E9B7
:10412000E7CFD9FF120000EBF6FF01EBF7FF12001B
:1041300045E9E7CFD9FF1200E552E5CFCDF1E7CF52
:10414000CCF11200E66EE66A46C2E6FF47C2E6FF21
:10415000D4EF2CF0C7EC35F048E9A2C2CCF1A3C2F1
:10416000CDF1A4C2CEF1A5C2CFF10101CE51120012
:1041700029DF400EE66EE66EB1EF1FF0CC272E0E63
:10418000CD23CCC1E6FFCDC1E6FFDFDC46E912005E
:10419000CCC1E6FF63DD44E90201462B000E472354
:1041A0001200400EE66EE66ADCDE200E5FEF20F0C5
:1041B0000E0EF6262E0EF7220900F550076E12009D
:1041C000E66EDACFE6FF1200E66EE66A00EBE6FF87
:1041D00001EBE6FF120020DF87E9120092EC2DF0E0
:0641E000ABDFC8EF20F088
:0A41E600800EC76E280EC66E180E7C
:1041F000C86EC56A800EE66E080EE66E8AEC3EF06A
:1042000042E90101636B646B006B016B010E026F8D
:10421000656B666B8A8A8996536B546B556B566BCC
:1042200053C14FF154C150F155C151F156C152F132
:1042300053C14BF154C14CF155C14DF156C14EF132
:10424000120056DB89E942E8010106500424CE6FD2
:1042500007500520CF6F0250CE25CC6F0350CF21E1
:10426000CD6FCC510024096ECD5101200A6E073468
:104270000550071804E60650045C0750055805E28F
:1042800006EBCEF107EBCFF104D004EBCEF105EB5A
:10429000CFF103340150031804E60250005C0350D0
:1042A000015805E202EBD0F103EBD1F104D000EBB1
:1042B000D0F101EBD1F1CF35CF51D11904E6CE5178
:1042C000D05DCF51D15913E207340550071804E6E9
:1042D0000650045C0750055805E206EBCCF107EBED
:1042E000CDF117D004EBCCF105EBCDF112D00334B6
:1042F0000150031804E60250005C0350015805E227
:1043000002EBCCF103EBCDF104D000EBCCF101EBEF
:10431000CDF1CC51095ECD510A5A0534075005182C
:1043200004E60450065C0550075805E206EBCEF1A2
:1043300007EBCFF104D004EBCEF105EBCFF1013464
:104340000350011804E60050025C0150035805E2D6
:1043500002EBD0F103EBD1F104D000EBD0F101EB93
:10436000D1F1D135D151CF1904E6D051CE5DD15123
:10437000CF5913E205340750051804E60450065CD3
:104380000550075805E206EBCCF107EBCDF117D04D
:1043900004EBCCF105EBCDF112D001340350011840
:1043A00004E60050025C0150035805E202EBCCF138
:1043B00003EBCDF104D000EBCCF101EBCDF1CC510E
:1043C000095ECD510A5A09EBCCF10AEBCDF1D89038
:1043D000CC37CD37CCC1F3FFCDC1F4FF43E9E7CFF4
:1043E000D9FF120085DA82E941E80050E824900FF5
:1043F000026EC7EC15F0A0EC3FF0C580C5B0FED74B
:1044000002EBE6FF8FDAC5AC02D0000E07D09F0E9C
:10441000E66E88DAC584C5B4FED7010EF36EF46A81
:1044200042E9E7CFD9FF120063DA84E946E8025097
:10443000E824910F046E800E076EC7EC15F0A0EC17
:104440003FF0C580C5B0FED704EBE6FF6BDAC5BC14
:1044500027D0030EE66ED950050FE66EDACFE6FFE1
:104460005DEC3DF043E9A0EC3FF0C58AC588C5B8D6
:10447000FED7C584C5B4FED705EBCEF1CEC1CFF1D2
:104480000101CE6B0650CE25CC6F000ECF21CD6F33
:1044900000EBE9FF01EBEAFF4ADA800E071402E0C5
:1044A000000E01D0010E47E9E7CFD9FF120020DA54
:1044B00082E90C0EE66E7F0E0014FE0BFD0BE66E1D
:1044C000AD0EE66E00EC3DF043E9010E35DAC9ECC5
:1044D0003FF041E9E7CFD9FF12000ADA81E942E86B
:1044E00079EC3FF0000EF35C016E020EF458026EA0
:1044F000C0EC3FF001EBF3FF02EBF4FF43E9E7CF41
:10450000D9FF1200020E1DDA030E1BDA010E19DAB2
:104510008F0EE66ECCDF41E91200EAD981E941E86D
:104520001EDA01E144D122DA01E141D126DA01E1CA
:104530003ED10101005113E05DC157F15EC158F158
:104540005FC159F160C15AF161C15BF162C15CF1B7
:104550008A9A030EF1D989860101006B24D1016A80
:10456000D890015002E6030E015C01E302D1F3D9B9
:10457000E9BEEA6890D9570EE926010EEA22EECF8D
:10458000D2F1EFCFD3F1E7D9E9BEEA6884D95D0E65
:10459000E926010EEA22EE500101D25DD06FEE5005
:1045A000D359D16FD06DD11F000ED123A6D9060EDD
:1045B000E926000EEA22ADD9CEBFCF698BD9E668D5
:1045C000E668E668E66863C1D4F164C1D5F1D66BEC
:1045D000D76BD5AF02D0D669D769D4C1E6FFD5C1B4
:1045E000E6FFD6C1E6FFD7C1E6FFB5D9E9BEEA6866
:1045F00052D951D93F0EE926010EA7D9EECFE6FFD9
:10460000EECFE6FF0DEC2DF0C6EC2DF0E552E5CF38
:10461000D3F1E5CFD2F1E5CFD1F1E7CFD0F16DD92C
:1046200078D9CEBFCF6956D996D9E9BEEA6833D9D1
:1046300032D94B0EE926010EEA22EE6AEE6AEE6AE4
:10464000EE6A89D9E9BEEA6826D9390EE926010E53
:104650001FD9E9BEEA681FD92D0EE926010E18D927
:10466000E9BEEA6818D9210EE926010E11D9E9BE82
:10467000EA6811D9150EE926010E16D9E9BEEA68D5
:10468000FD0EE926000EEA22EFCFCEF10101CF6B3D
:10469000CEBFCF6912D9E9BEEA68FDD8090EE92676
:1046A000010EEA2244D957D9E9BEEA68F4D8330E9C
:1046B000E926010EEDD8E9BEEA68EDD8270EE92615
:1046C000010EE6D8E9BEEA68E6D81B0EE926010E1F
:1046D000DFD8E9BEEA68DFD80F0EE926010EE4D87C
:1046E000E9BEEA68FA0EE926000EEA22EFCFCEF123
:1046F0000101CF6BCEBFCF69E0D8E9BEEA68CBD865
:10470000030EE926010EEA2212D90001C751800BDF
:1047100027E021D9E9BEEA68BED8090EE926010ED4
:1047200014D9FDEC36F042E9F3CFCCF1F4CFCDF162
:10473000140E0101D890CDBF03D0CC5D000ECD5931
:104740000FE2010E01EBF3FF015204E0D890E836CE
:10475000F306FCE101016511656F030E662707D0C2
:104760000101665102E0660501D0000E666F012A64
:10477000F7D6665101E1656B8996030EDDD88A8A0A
:104780000101010E006F030EE66E010EE66E0BECEA
:1047900025F042E90101636B646B022B02510408AE
:1047A00002E2010E026FAEDE0101016B19D00101C0
:1047B000643516E263516408000E645511E2100E70
:1047C000656FCDD802E101016581D0D802E1010118
:1047D0006583D3D802E10101658501010A0E666F88
:1047E000B8EC3FF0000950E178DEF3CFCCF1F4CF24
:1047F000CDF10101CE6BCF6BCDAF02D0CE69CF69C9
:1048000001010151040DF3CFE9FFF4CFEAFF4B0E94
:10481000E926010EEA220101CC51EE26CD51EE220D
:10482000CE51EE22CF51EE220101012B030E015D8C
:104830001CE3016B4BC13FF14CC140F14DC141F153
:104840004EC142F14FC143F150C144F151C145F154
:1048500052C146F153C147F154C148F155C149F124
:1048600056C14AF1632B000E64230151020A08E08D
:10487000030A04E0010A08E18F0E03D0970E01D06D
:10488000870EE66E14DE41E942E9E7CFD9FF120058
:104890005CD8ABEF24F0D890E936EA361200E66E29
:1048A000C3DD43E90009120050D8CBDC48E9F3CF5F
:1048B000E6FFF4CFE6FFABEF24F0CEC1E6FFCFC1B9
:1048C000E6FF92EC2DF0E552E5CFCDF1E7CFCCF14C
:1048D000ABEF24F0D890CE37CF37CC51CE25E96E50
:1048E000CD51CF21EA6ED0C1EEFFD1C1EDFF120054
:1048F000D9CFE6FFE1CFD9FF1200010102510C0D23
:10490000F3CFE9FFF4CFEAFF030EE926010EEA2216
:104910001200E9CFCCF1EACFCDF101EBCEF10101EC
:10492000CF6B1200B1EC3DF041E9A0EF3FF0CCC1FC
:10493000EEFFCDC1EDFF1200E66E85EC3FF041E9E0
:104940001200E66E4FDD41E91200EA22EECFE6FFEB
:10495000EECFE6FF120001EBE9FFEA6A12005D0EFE
:10496000E66E010EE66E020E4FEF24F05F0EE66E6D
:10497000010EE66E030E4FEF24F0610EE66E010E9F
:08498000E66E010E4FEF24F07A
:08498800D6DA83E941E8036A75
:10499000D890035002E6180E035C39E2040EE66E6E
:1049A00003EBE6FF6EEC2DF041E9E750000906E06D
:1049B0000101D06BD16BD26BD36B06D00101D06BF0
:1049C000D16BD26B010ED36F00EBE9FF01EBEAFF75
:1049D000E9CFCCF1EACFCDF103EBCEF1CF6BCEBF77
:1049E000CF69D890CE37CF37D890CE37CF37CC518C
:1049F000CE25E96ECD51CF21EA6ED0C1EEFFD1C1F7
:104A0000EEFFD2C1EEFFD3C1EEFF032AC1D742E9C8
:104A1000E7CFD9FF12008FDA83E945E8036AD8901F
:104A2000035002E6060E035C0EE203EBE9FFEA6ABE
:104A3000E9BEEA68A8DA03EBE9FFEA6AE9BEEA68D8
:104A4000A5DA032AECD7E66A00EBE6FF01EBE6FF06
:104A500022EC0CF043E92CC2CCF12DC2CDF12EC2D8
:104A6000CEF12FC2CFF1020130510101CC2702015A
:104A700031510101CD23020132510101CE23020146
:104A800033510101CF233CDA06DA73EC36F044E906
:104A900049DA0ADA00DA58DAE5D9010131DA39DA25
:104AA00014C2E6FF15C2E6FF16C2E6FF17C2E6FF14
:104AB00018C2E6FF19C2E6FF1AC2E6FF1BC2E6FFF4
:104AC00054DAA2C200F2A3C201F2A4C202F2A5C249
:104AD00003F20201033504E3680E0227010E0323EB
:104AE00018DAD9D91CC2E6FF1DC2E6FF1EC2E6FFD6
:104AF0001FC2E6FF3ADAA2C204F2A3C205F2A4C2C0
:104B000006F2A5C207F246E9E7CFD9FF120013DA91
:104B100081E94CE8056A066A076A086A0A6A0B6A4C
:104B2000060ED8900BBE03D00A5C000E0B580EE2A6
:104B30000AEBE9FF0BEBEAFF26DA0AEBE9FF0BEBE6
:104B4000EAFF24DA0A2A000E0B22EAD70A6A0B6A65
:104B5000380ED8900BBE03D00A5C000E0B5801E350
:104B60008CD00AEBE6FF0AEBCEF10BEBCFF10101A3
:104B70000C0ECF03F3CFCFF1CE03F3CFCEF1F45031
:104B8000CF27020188510101F324CC6F0201895122
:104B90000101CF21CD6FCCC1E6FFE66E22EC0CF017
:104BA00043E9100ED8900BBE03D00A5C000E0B58E0
:104BB00060E2030E01010A14CC6FCD6B030ECC1919
:104BC00058E1CD5156E1096AD890095002E6030E2A
:104BD000095C4FE2020EE66EE66AE66AE66AB0D962
:104BE000E9BEEA6833D9C8D9EFCFE6FF0DEC2DF066
:104BF000E552E5CFEDFFE5CFEDFFE5CFEDFFE7CFE8
:104C0000EFFF9ED9E9BEEA6821D9EE50016EEE5061
:104C1000026EEE50036EEF50046E92D9E9BEEA6860
:104C2000BDD98ED9E9BEEA6893D901EBD0F102EB88
:104C3000D1F103EBD2F104EBD3F182D9E9BEEA68FA
:104C40000BD944D9D950050FE96EDACFEAFFCC5120
:104C5000EE26CD51EE22CE51EE22CF51EE2270D96A
:104C6000E9BEEA6893D96CD9E9BEEA688CD9092A09
:104C7000ABD70A2A000E0B226BD7030E0C6ED8900E
:104C80000C5002E6060E0C5C47E2EDC1E6FFEEC1F9
:104C9000E6FFEFC1E6FFF0C1E6FF0CEBE9FFEA6AD1
:104CA000E9BEEA6855D90CEBE9FFEA6AE9BEEA68B1
:104CB00075D901EBE6FF02EBE6FF03EBE6FF04EB41
:104CC000E6FF42D92FD90CEBE9FFEA6AE9BEEA68B0
:104CD000C3D80101FBD8F1D8D950010FE96EDACF62
:104CE000EAFF020EE76ED890030EEB32020EEB32B3
:104CF000010EEB32EF32E706F6E1D950050FE96E0F
:104D0000DACFEAFF0150EE260250EE220350EE22E7
:104D10000450EE220C2AB3D705EBA2F206EBA3F265
:104D200007EBA4F208EBA5F24DE9E7CFD9FF12009B
:104D300030D92ADE42E99FD8EADEA2C20CF2A3C231
:104D40000DF2A4C20EF2A5C20FF20201106B116B9C
:104D5000200E126F136B1200EED882E945E80201B3
:104D6000105111111211131165E0005002E1010EF2
:104D7000456F066AD890065002E6180E065C4AE2B5
:104D80007AD800500EE006EBE9FFEA6AE9BEEA686D
:104D9000AAD8EE261151EE221251EE221351EE2224
:104DA0000DD006EBE9FFEA6AE9BEEA689CD8EE5E40
:104DB0001151EE5A1251EE5A1351EE5AA8DE52D842
:104DC0000101CC51026ECD51036ECE51046ECF5114
:104DD000056E02010C51025C0D5103580E5104582E
:104DE0000F51055815E2600EE66EE66A600EE66E3B
:104DF000000EE66ECED88BEC34F046E902EB0CF2F6
:104E000003EB0DF204EB0EF205EB0FF20201456B22
:104E1000062AB0D745510DE000500BE0010E1F0BE4
:104E200008E00201D8901333123311331033E8062F
:104E3000F9E121D80CC2A2F20DC2A3F20EC2A4F273
:104E40000FC2A5F246E9E7CFD9FF120087D8140EAA
:104E5000E926020EEA22120081D82C0EE926020E63
:104E6000EA221200A2C2CCF1A3C2CDF1A4C2CEF1BB
:104E7000A5C2CFF11200600EE66EE66A8AD8600E17
:104E8000E66E000EE66E8BEC34F046E9120074D844
:104E9000EECFE6FF120004EBE6FF05EBE6FF06EBC4
:104EA000E6FF07EBE6FF1200A2C2E6FFA3C2E6FFA1
:104EB000A4C2E6FFA5C2E6FF1200CC51016ECD519F
:104EC000026ECE51036ECF51046E1200D051EE5CD3
:104ED000CC6FD151EE58CD6FD251EE58CE6FD35129
:104EE000EE58CF6F12003AD8600EE926000EEA2283
:104EF000020110511200EE6AEE6AEE6AEE6A1200CA
:104F0000CC51046ECD51056ECE51066ECF51076E59
:104F10001200E9C1E6FFEAC1E6FFEBC1E6FFECC122
:104F2000E6FF1200A2C2D0F1A3C2D1F1A4C2D2F115
:104F3000A5C2D3F11200D9CFE6FFE1CFD9FF12000D
:104F400009EBE9FFEA6A1200C7EC35F048E9120004
:104F500025D8FADF87DF01015DEF27F0D890E93629
:104F6000EA36D890E936EA361200A5EC2AF048E98C
:104F700079DF9ADFA4EF27F0EECFE6FFEECFE6FF72
:104F8000EECFE6FF120062DF7BEF27F065DF7BEFFD
:104F900027F0A00EE66E070EE66E120057DF47EF11
:024FA00027F0F8
:0E4FA200060EE66E70EC3EF041E9400EE66E43
:104FB000D1EC3CF041E9D70E9314936E99EC3FF09D
:104FC000BA6A8A86670EE66EE66A3C0EE66EC1EC49
:104FD0003BF043E9E60EE66E4BEC3FF041E9E10EB3
:104FE000E66E740EF6D9BE0EE66E740EF2D9B10EF0
:104FF000E66E740EEED9A20EE66E740EEAD99D0E20
:10500000E66E740EE9EF29F0F3D987E9960EE66EA5
:10501000740EE66EE66A1BDA47EC35F045E9D9CF47
:10502000E9FFDACFEAFF080EE76ED890030EEB3205
:10503000020EEB32010EEB32EF32E706F6E1E4D975
:10504000E3D9BED9C7EC35F048E9A2C2D0F1A3C27A
:10505000D1F1A4C2D2F1A5C2D3F1A2C2E6FFA3C28C
:10506000E6FFA4C2E6FFA5C2E6FFC7EC35F048E9BB
:10507000A2C2CCF1A3C2CDF1A4C2CEF1A5C2CFF1A0
:10508000A4C2E6FFA5C2E6FF050EE66EE0D950EC2D
:1050900037F045E9080E7FD9EF6A070E7CD92C0E50
:1050A000EF6E050E78D9EF50E66E060EC9D9EF50B7
:1050B000E66E050EC5D92E0EEF6E41E9E7CFD9FF9A
:1050C000120096D98BE956E80B6A97D90D0FADD926
:1050D00077D9D950170FA9D98C0EE66E740EA9D9BD
:1050E00047EC35F045E9D9500D0F79D9D950170F54
:1050F00076D9860EE66E740E9CD917EC35F045E92C
:10510000010E0C6E0CEBCCF10101CD6BCCBFCD6967
:1051100084D92A080AE00CEBCCF1CD6BCCBFCD6969
:105120007CD90B180B6E0C2AEDD7E66AD9500B0F01
:1051300093D9010EE66E0CEBCEF1CF6BCEBFCF69EB
:105140000850CE25CC6F0950CF21CD6FCC2B000E4F
:10515000CD23CCC1E6FFCDC1E6FF75EC37F046E9C3
:1051600057E9E7CFD9FF120043D989E972E828D976
:1051700044D9090F71D9A5DF4AE9D950090F6CD973
:10518000D7EC3DF042E973E9E7CFD9FF120030D9FF
:1051900082E9005003E00C0EBA6E02D0BA6A8A8629
:1051A0000028E86CE66EE66A8BEC3DF042E941E9E6
:1051B000E7CFD9FF12001CD983E946E8CE0E036E73
:1051C000720E046E050EE66EE66A200E015C0101A9
:1051D000CC6FCD6B800B01E0CD69CCC1E6FFCDC1BA
:1051E000E6FF92EC2DF0E552E550076EE750066EB3
:1051F000056A050E055C2EE2005022E0040ED88000
:105200000554CFD8086E700E0814E8380F0BCD6F18
:10521000070E0814100D080E0814F310CD11086EB7
:10522000440E0814E840E8403F0BCD6F110E0814FF
:10523000040DF3CFCCF12A0E0814F310CD1102D0D7
:105240000550AFD8086E08EBE6FFA2EC3CF041E950
:10525000052ACFD747E9E7CFD9FF1200D9CFE6FF1C
:10526000E1CFD9FF83E942E8C7EC15F00201D8800D
:105270000B5104E7C00E0A5DFF0E0B5901E2046AF0
:1052800002010B3504E20A514008000E0B5502E200
:10529000010E046E0001C7AB04D0010ED880045487
:1052A000046E0001CA5102E1899855D0040EE66EE1
:1052B000E66A00EBE6FF01EBE6FFF50EE66E010E97
:1052C000E66E6EEC35F046E9000945E0050EE66E47
:1052D000E66A00EBE6FF01EBE6FFF50EE66E010E77
:1052E000E66E99EC35F046E989980000898800005F
:1052F000CAC0E6FF34D841E900008B9200008B80E1
:105300000000C7EC3FF00000036A040E035C1EE2DD
:1053100004500FE0010EE66E030ED8800354002403
:10532000E96E000E0120EA6EEFCFE6FF44DF42E9AE
:105330000BD0E66A03500024E96E000E0120EA6EED
:10534000EFCFE6FF38DF42E9032ADFD70000C3ECE6
:105350003FF000008B9043E9E7CFD9FF1200D9CF8F
:10536000E6FFE1CFD9FF82E98B8200008B8000004D
:10537000C7EC3FF00000400E00107F0BE66EA2EC81
:105380003CF041E90000C3EC3FF000008B9041E9A4
:10539000E7CFD9FF12000424E96E000E0520EA6E63
:1053A000120001010624CC6F000E0720CD6FCC51F6
:1053B0000324F66ECD510420F76E0800F55012005C
:1053C00000EBE6FF01EBE6FF02EBE6FF03EBE6FF97
:1053D0001200E66EE66A2FEC3DF043E912003CD87D
:1053E00008EBE6FF09EBE6FFF3EC34F044E91200CA
:1053F000D9CFE6FFE1CFD9FF120029D806EBE6FFAF
:1054000007EBE6FFD9501200E0C1E6FFE1C1E6FF7D
:10541000E2C1E6FFE3C1E6FF1200CC510824E96EC9
:10542000CD510920EA6EEF50120016D8EDDD46E9A5
:105430001200E66EE66A08EBE6FF09EBE6FF1200F3
:10544000AADFE552E750EF6E040ECBEF29F004EB34
:10545000E6FF05EBE6FF1200E66EDACFE6FF12008C
:1054600005DA89E945E807340CE3C8D993D97BD933
:10547000046ECD51056ECE51066ECF51076E010EF2
:105480000D6E03340CE327DA006ECD51016ECE5160
:10549000026ECF51036E010ED8800D540D6E02EBDB
:1054A000D0F103EBD1F10101D26BD36BD1AF02D0BC
:1054B000D269D369D0C1E6FFD1C1E6FFD2C1E6FF10
:1054C000D3C1E6FF67D90DEC2DF0E9D9080E1F0B0B
:1054D00008E00101D890CC37CD37CE37CF37E8067A
:1054E000F9E10101CC5171D90D5001E0E2D909EB8C
:1054F000A2F20AEBA3F20BEBA4F20CEBA5F246E945
:10550000E7CFD9FF1200B2D985E944E8033409E2B4
:1055100000EBA2F201EBA3F202EBA4F203EBA5F283
:1055200010D0D9D9056ECD51066ECE51076ECF5130
:10553000086E05EBA2F206EBA3F207EBA4F208EB70
:10554000A5F245E9E7CFD9FF120090D989E959E8DA
:10555000216A20D9D8DF44E9B1D9A2C2E6FFA3C2AB
:10556000E6FFA4C2E6FFA5C2E6FF1DD9CCDF44E9F1
:10557000E552E7CFCFF1E552E7CFCEF1E552E7CFE5
:10558000CDF1E552E7CFCCF1A2C2D0F1A3C2D1F167
:10559000A4C2D2F1A5C2D3F10101D335CF51D319A1
:1055A00008E6D051CC5DD151CD59D251CE59D3510D
:1055B000CF5904E3EFD8F7D892D905D0F4D8EAD878
:1055C0008ED9010E216E0C3401E373D9D2D8D1D813
:1055D00090D90D6ECD510E6ECE510F6ECF51106E13
:1055E0001CD9950ECC27DB0ECD23020ECE23F90E4F
:1055F000CF23CC51FBD8690E156E1F0E166EF30E1D
:10560000176E186813D948D9BDD807D9050ECC270D
:10561000000ECD23CE23CF23CC51E8D807D957D9BC
:10562000F30E156E8E0E166ED30E5DD908D9CA0E06
:10563000CC272E0ECD23D80ECE23020ECF230DEB7A
:10564000D0F10EEBD1F10FEBD2F110EBD3F1DBD8AF
:1056500005D9B2D83CD99B0E156EA80E166E250E34
:1056600042D9540E156EFB0E166EA40E176E186AF4
:105670000DEBE6FF0EEBE6FF0FEBE6FF10EBE6FFB0
:105680000BD9ECD8DCD8CF2B15EBD0F116EBD1F140
:1056900017EBD2F118EBD3F1B6D8196ECD511A6EC3
:1056A000CE511B6ECF511C6E19EBE6FF1AEBE6FFD5
:1056B0001BEBE6FF1CEBE6FF90D8D2DE4FD862D89A
:1056C000215012E1203408E2B50ED06F1F0ED16FC9
:1056D000920ED26F010E07D04B0ED06FE00ED16F3D
:1056E0006D0ED26FFE0EC7D807340DE204500008CD
:1056F000000E0554000E0654000E075404E27ED836
:105700006CD831D83FD8033408E3960ED06FC00E62
:10571000D16FDB0ED26FFC0EAED8D880205008E7D8
:10572000960E1D5CC00E1E58DB0E1F58FC0E205836
:1057300009E28ED8D40EEE267E0EEE22480EEE2220
:10574000060EEE221DEBA2F21EEBA3F21FEBA4F25B
:1057500020EBA5F25AE9E7CFD9FF120048E9AED80D
:105760000101CC511200C6EC2DF099D80101CC51A9
:10577000120009EBE6FF0AEBE6FF0BEBE6FF0CEB92
:10578000E6FF12001D6ECD511E6ECE511F6ECF5121
:10579000206E120004EBE6FF05EBE6FF06EBE6FFEA
:1057A00007EBE6FF120000EBE6FF01EBE6FF02EB82
:1057B000E6FF03EBE6FF120015EBE6FF16EBE6FF54
:1057C00017EBE6FF18EBE6FF1200096ECD510A6EEB
:1057D000CE510B6ECF510C6E12001DEBE6FF1EEB8F
:1057E000E6FF1FEBE6FF20EBE6FF1200116ECD5146
:1057F000126ECE51136ECF51146E1200E668E66839
:10580000E668E6681200D051CC27D151CD23D251A1
:10581000CE23D351CF23CC51120009EBCCF10AEBAC
:10582000CDF10BEBCEF10CEBCFF1120011EBE6FF5B
:1058300012EBE6FF13EBE6FF14EBE6FF120011EBB1
:10584000CCF112EBCDF113EBCEF114EBCFF1120052
:10585000D9501D0FE96EDACFEAFF1200156ECD5157
:10586000166ECE51176ECF51186E1200D9CFE6FFCB
:10587000E1CFD9FF1200D36FEBDFEE50D05DCC6FDC
:10588000EE50D159CD6FEE50D259CE6FEE50D35964
:10589000CF6FCC51C2EF2BF08FDF79EF2CF0E552B8
:1058A000E5CFCFF1E5CFCEF1E5CFCDF1E7CFCCF12C
:1058B0001200A4DF5EDF57DFE5EF2BF0A2C2CCF1D0
:1058C000A3C2CDF1A4C2CEF1A5C2CFF1120085DFF3
:1058D00010D8C2EF2BF092DF66DFB3EF2BF0C0DD04
:1058E0003DDFE5EF2BF0176E186A43DFD5DFF6EFEB
:0A58F0002BF0C7EC35F0AEEF2BF003
:0658FA0043E8D9CFE6FFF0
:10590000DACFE6FFE1CFD9FFE2CFDAFF89E9066A15
:105910001200F3DF068001D0F0DF01AE96EF2CF02D
:10592000006C011EE86A012206B0067E03AE9EEFFF
:105930002CF0026C031EE86A0322067ED6EC2CF0E3
:1059400003BEC0EF2CF006AE08D0026C031EE86A5E
:105950000322046C051EE86A052206B006D084EB1B
:1059600000F085EB01F006A004D082EB00F083EBA1
:1059700001F0E552E5CFDAFFE7CFD9FF45E9000CAA
:1059800006BEA5EF2CF0E9DFFF0C43E8D9CFE6FF18
:10599000DACFE6FFE1CFD9FFE2CFDAFF89E9066A85
:1059A0001200F3DF068003D0F0DF01D00682056A23
:1059B000046A100EE76ED8900236033604360536B8
:1059C0000050045C0150055805E30050045E01508E
:1059D000055A022AE72EF0D706B2120006B006D00A
:1059E00084EB00F085EB01F006A004D082EB00F020
:1059F00083EB01F0E552E5CFDAFFE7CFD9FF45E9C8
:105A0000120045E8D9CFE6FFDACFE6FFE1CFD9FFB4
:105A1000E2CFDAFF8FE90C6A1200F3DF0C8001D0CD
:105A2000F0DFE86A03AE1EEF2DF0006C011E021ECF
:105A3000031E0122022203220CB00C7E07AE29EFC6
:105A40002DF0046C051E061E071E052206220722E5
:105A50000C7E56EC2EF007BE5AEF2DF00CAE0FD098
:105A6000046C051E061E071EE86A05220622072290
:105A7000086C091E0A1E0B1E09220A220B220CB0FA
:105A80000AD088EB00F089EB01F08AEB02F08BEB97
:105A900003F00CA008D084EB00F085EB01F086EB5E
:105AA00002F087EB03F0E552E5CFDAFFE7CFD9FF4D
:105AB00049E9000C0CBE30EF2DF0E1DFFF0C42E8AD
:105AC000D9CFE6FFDACFE6FFE1CFD9FFE2CFDAFFA9
:105AD00086E9036A1200F3DF038001D0F0DF00AE35
:105AE00003D0006C03B0037E01AE02D0016C037ED4
:105AF00028EC2EF001BE8EEF2DF003AE02D0016C2B
:105B0000026C03B081EB00F003A082EB00F0E552E1
:105B1000E5CFDAFFE7CFD9FF43E9000C03BEEFD7AB
:105B2000F0DFFF0C44E8D9CFE6FFDACFE6FFE1CFA4
:105B3000D9FFE2CFDAFF8AE980EB04F081EB05F0D0
:105B400082EB06F002500402F450016EF350006E36
:105B50000350076E0502F450036EF350026E0750B7
:105B60000402F3500126F4500222E86A0322065090
:105B70000502F3500126F4500222E86A0322E5529E
:105B8000E5CFDAFFE7CFD9FF46E9000C44E8D9CFEB
:105B9000E6FFDACFE6FFE1CFD9FFE2CFDAFF8EE909
:105BA00080EB08F081EB09F082EB0AF083EB0BF05D
:105BB00004500802F350006EF450016E04500902C4
:105BC000F3500126000EF420026E04500A02F35036
:105BD0000226000EF420036E04500B02F35003263D
:105BE00005500802F3500126F4500222000E032251
:105BF00005500902F3500226F450032205500A0210
:105C0000F350032606500802F3500226F4500322F4
:105C100006500902F350032607500802F3500326EA
:105C2000E552E5CFDAFFE7CFD9FF48E9000C42E8BB
:105C3000D9CFE6FFDACFE6FFE1CFD9FFE2CFDAFF37
:105C400086E9036A1200F3DF038003D0F0DF01D09E
:105C50000382026A080EE76ED890013602360050C1
:105C6000025C02E3026E012AE72EF7D703B21200AC
:105C700003B081EB00F003A082EB00F0E552E5CF2A
:105C8000DAFFE7CFD9FF43E9120045E8D9CFE6FFB5
:105C9000DACFE6FFE1CFD9FFE2CFDAFF8FE90C6A76
:105CA0001200F3DF0C8003D0F0DF01D00C820B6A0E
:105CB0000A6A096A086A200EE76ED890043605362B
:105CC00006360736083609360A360B360050085CA9
:105CD0000150095802500A5803500B5809E300506C
:105CE000085E0150095A02500A5A03500B5A042AFE
:105CF000E72EE4D70CB212000CB00AD088EB00F00B
:105D000089EB01F08AEB02F08BEB03F00CA008D0DA
:105D100084EB00F085EB01F086EB02F087EB03F0FB
:0E5D2000E552E5CFDAFFE7CFD9FF49E91200DF
:025D2E00020E63
:105D3000E66EF20EE66E9D0EE66E020EE66E43EC29
:105D40001EF044E99DC29FF29EC2A0F21200200EF6
:105D5000E66E310E67D9440EE66EFE0E63D9020E72
:105D6000E66E5CEC3FF041E9B40EE66EFE0E5AD9E9
:105D700087D902019D6BF60E9E6F1EEF30F059D948
:105D800082E944E8046A056A020EE66ED950020F01
:105D9000E66EDACFE6FF00EBE6FF680EE66E29EC72
:105DA0003BF045E9000913E1FF0E01010214CD6B40
:105DB000CD6FCC6B000E0214FF0E0314CF6FCE6FAD
:105DC000CF6BCE51CC11046ECD51CF11056E04EBCB
:105DD000F3FF05EBF4FF5AD1E66A010EE66E180EEA
:105DE00070D9F3CFE6FFF4CFE6FF89EC2CF0E55253
:105DF000E5CFCDF1E7CFCCF1CCC1F3FFCDC1F4FFBE
:105E0000120017D981E948E845D9056AC00E066E27
:105E1000076A086A0E0E28D905EBE6FF06EBE6FFD7
:105E200007EBE6FF08EBE6FFEAD849E9E7CFD9FF41
:105E30001200FFD881E944E82DD90C0E15D9AAC269
:105E4000E6FFABC2E6FFACC2E6FFADC2E6FFD7D8C5
:105E50001DD1100E61EF30F0ECD883E9010101EBA8
:105E6000CCF1CD6BCCC1E6FF100EDCD800EBE6FF29
:105E7000110ED8D841E9E7CFD9FF1200800EE66EA7
:105E8000080ED0D8E7D801E0000C010CD2D881E987
:105E900044E8DFDFEFD8CE6BCF6BCDAF02D0CE6959
:105EA000CF69FDD89DC2CCF19EC2CDF1CE6BCF6B38
:105EB000CDAF02D0CE69CF69CF350450CF1908E6F7
:105EC000CC51015CCD510258CE510358CF510458EA
:105ED00004E201EB9DF202EB9EF2ABDFCBD8D8904F
:105EE000F45004E6800ECC5D0C0ECD5907E201EBB8
:105EF0009DF202EB9EF20201A1693BD0043401E263
:105F0000C9D8640ED06FD16BD26BD36B9DC2D8F160
:105F10009EC2D9F1DA6BDB6BD9AF02D0DA69DB69EB
:105F2000D8C1E6FFD9C1E6FFDAC1E6FFDBC1E6FF73
:105F3000E66EE66AE66AE66ABBD8C6EC2DF00DECC2
:105F40002DF0E552E5CFD7F1E5CFD6F1E5CFD5F18C
:105F5000E7CFD4F10101D451D05DCC6FD551D159E7
:105F6000CD6FD651D259CE6FD751D359CF6FCCC147
:105F7000A1F28CD05ED882E941E8E66AC7EC28F04D
:105F800041E9E66AAFEC29F041E9005008E0E66A31
:105F90003AEC3EF041E9E66A3AEC3EF041E95AD883
:105FA00021E002019F519D1902E1A0519E1901E0DB
:105FB00045D84FDF5FD8F43406E2CC510008000E1C
:105FC000CD5501E25DD8E668AA0EE66EF9EC1DF04B
:105FD00042E9C5EC3FF093909392080E8A6E816E71
:105FE000D190FFD7E668C7EC28F041E93F0EE66E96
:105FF000AFEC29F041E942E9E7CFD9FF120058D8C8
:10600000C7EC35F048E9A2C2CCF1A3C2CDF1A4C2DD
:10601000CEF1A5C2CFF1010142D803EBF3FF04EBAF
:10602000F4FF1200E66E680EE66E02EC3CF043E907
:106030001200D9CFE6FFE1CFD9FF1200020EE66EC3
:106040009D0EE66E020EE66EF20EE66E2EEC1EF071
:1060500044E91200080EE66E680EE66E76EC3BF040
:1060600042E9F350800B12002CD8F350036EF45029
:10607000046E1200F3CFCCF1F4CFCDF10101120088
:10608000000EE66EE66AE8DE42E9120045E9E7CF77
:10609000D9FF1200016A026A036A046A1200CC5135
:1060A000016ECD51026ECE51036ECF51046E1200BF
:1060B00001EBE6FF02EBE6FF03EBE6FF04EBE6FF96
:0A60C0001200E66E5CDE41E91200FA
:0660CA006C5007E168962E
:1060D00067D902E10AD8010C37D8010C040E6C5CB8
:1060E00003E1689640D8010C000C54D941E8040142
:1060F00004BF046B02019C6B946B956B9A6B9B6B5A
:106100004AEC33F0016A010E52D919E202019551AD
:1061100016E1F76A0134FE0BF66EF736B20EF6267C
:10612000750EF7220900F5CFCCF10800F5CFCDF1BF
:10613000CDC1FAFF0101CC511400012AE4D7A3D844
:1061400042E9E7CFD9FF1200020E0201945D09E196
:1061500070D8040100BD02D0C80E01D0880E006FB7
:1061600012007CEF31F0040E0201A65D09E122C4A9
:106170006EFF6E50000802E2050E01D0030EA66FFE
:106180000201940510E111D8020E02019C5D03E1A9
:106190000401840E06D0040104BD02D0C80E01D053
:1061A000880E046F12007CEF31F0F4D842E802014F
:1061B000200E9A5D000E9B590DE29A51016E9B5183
:1061C000026E9C5102E1010E03D09C0506E1020E15
:1061D0009C6F03D0200E016E026A040104930491A7
:1061E0000250041301EB05F4015002019A5F0250C2
:1061F0009B5B400E986F040E996F0201A7A30BD012
:106200000150021012E096C2F6FF97C2F7FF080095
:10621000F550B0D8F5D70150021007E096C2E9FF5B
:1062200097C2EAFFEF50A6D8F6D743E9E7CFD9FFE8
:106230001200B0D842E8030E04010015026E0151AD
:10624000016E9A0EE96E020EEA6E0201EE50012412
:106250009A6FED5002209B6F400E966F040E976F61
:10626000015002100CE096C2E9FF97C2EAFFEF501E
:1062700098C2E9FF99C2EAFFEF6EA0D8F1D743E9CF
:10628000E7CFD9FF12006D980201955105E17AD848
:10629000840E006F04011DD0040120AF1CD0020148
:1062A0009A510401265D02019B510401275904E221
:1062B00026C49AF227C49BF278DF0201010E946F84
:1062C00061D8800E006F0401400E066F040E076F48
:1062D000C80E046F12000201020E946F0401056BD8
:1062E000C80E046F0401200E016F400E026F040EF1
:1062F000036FC80E006F12004DD841E8020E020174
:10630000945D2DE16D50100B2AE004010151010153
:10631000CC6FCD6B200ECC1922E1CD5120E140D8BD
:106320001EE10051800B1BE1200E026F040E036F73
:10633000016A200E3CD81AE20150EA6A400FE96E69
:10634000040EEA22EF50E66E0150EA6A200FE96E71
:10635000040EEA22E552E750EF6E012AEAD7020165
:10636000946B10D88C0E006F0401046B42E9E7CFE8
:10637000D9FF120098C2E9FF99C2EAFFEF6E02014D
:10638000DEEF31F00401200E016F200E026F040ECB
:10639000036F1200D9CFE6FFE1CFD9FF81E91200E8
:1063A000040100513C0BE842E8420D081200F36E74
:1063B000F46AF350015C000EF4541200982B000EA6
:0C63C0009923962B97230106025A120025
:0463CC000401205157
:1063D0001F0B010801E012002051600BE842E84267
:1063E000E842E842E842010801E01200245103E0DB
:1063F000240501E012002151230A39E0010A33E0AB
:10640000030A25E0010A1CE0240A31E0070A2FE014
:10641000010A2DE0030A0EE0010A01E0120031D961
:106420000201F20E966F000E976F0201A793020110
:10643000080E17D026D90201F20E986F000E05D073
:1064400020D90201EA0E986F000E996F120019D937
:106450000201EA0E966F000E976F0201A7930201E8
:10646000070E9A6F12000DD922C4F1F0120012002B
:106470000001EA6BC20EEB6F010EEC6FED6BEE6B81
:10648000EF6B080EF06FE36BE26B1A0E726E1E0E6E
:10649000736E0401600E166F040E176F400E146FBA
:1064A0000401196F680E1A6F040E1B6F880E186FA7
:1064B0000401A80E1E6F040E1F6F400E1C6F120009
:1064C000E4D884E90001E26B040118BF24D0005035
:1064D000195D02E21951006E0001E26B0050E25DAD
:1064E00013E2E251EA6A680FE96E040EEA22EF5005
:1064F000E66EE2510124E96E000E0220EA6EE552DA
:10650000E750EF6EE22BEAD70401400E196F18171F
:10651000187D880E18130001E25141E9E7CFD9FF39
:1065200012009ED812E1036AA1D802E1F45009E0FA
:1065300000EBE9FF01EBEAFF002A000E0122EF5019
:10654000F3E176D8E96B010EE36F97D089D813E1B8
:10655000036A8CD802E1F4500AE000EBF6FF01EB8D
:10656000F7FF002A000E01220800F550F2E160D882
:10657000010EE96FE36F81D088D881E941E8040119
:106580001CBF55D0030E0001E35D01E1E36BE35155
:106590004EE0020EE35D03E104011D6B3FD0E30515
:1065A00040E1E8510101CC6FCD6BCC514008000EA9
:1065B000CD5502E2400E02D00001E851016E01EB20
:1065C0001DF401500001E85DE86FA80EE66F040EAF
:1065D000E76FE9050AE1015011E0E4C0F6FFE5C00C
:1065E000F7FF0800F55030D8F6D7015007E0E4C0B7
:1065F000E9FFE5C0EAFFEF5027D8F7D70001E851DF
:1066000010E104011D510101CC6FCD6B400ECC197E
:1066100005E1CD5103E10001020E02D00001030E9D
:10662000E36F400E04011C171C7D880E1C1325D03F
:106630000350005E000E015A00EBE4F001EBE5F0C0
:1066400003EBE8F000011200E6C0E9FFE7C0EAFF53
:10665000EF6EE62B000EE723E42BE5230106120084
:1066600014D883E941E80001E3511200032AFF0E28
:10667000F36EF46AF3500318120042E9E7CFD9FF32
:1066800012000201030E956F1200D9CFE6FFE1CF91
:04669000D9FF12001C
:0C66940004012051600BE842E842E8429B
:1066A000E842E842000901E012002151070A3FE0F8
:1066B0000B0A3DE0070A32E0010A23E00B0A1FE063
:1066C000020A1DE0030A19E0080A10E0010A0CE0C2
:1066D0000F0A08E0030A01E0120015D90201040EB6
:1066E000A66F120098EF33F0CFEF33F00CD9020110
:1066F000A80E966F020E976F0BD0F0EF33F022EFDB
:1067000034F005D90201976BA90F966F020E9723FB
:106710000201A7930201010E9A6F1200F8D8EA6AEB
:10672000A90FE96E020EEA2222C4EFFF1200120046
:10673000800E0401205D32E12351030A1FE0010AAB
:106740000AE0030A29E1DFD80201E70E966F740E12
:10675000976F120E1ED0C6D8A80EF626750ECBD88F
:10676000020E0201F76A9625F66E9751F72209008C
:10677000F5CF9AF20A00F5CF9BF20ED0B3D8AC0E4B
:10678000F626750EB8D896C2F6FF97C2F7FF080036
:10679000F55002019A6F9B6B0201A7831200B3D8D8
:1067A0000F0EE66E710EE66E0F0EE66EBBEC38F065
:1067B00043E9010EE66EA90EE66E020EE66EBBEC34
:1067C00038F043E922C4A8F20401225104E1020195
:1067D000050EA66F12000201060EA66F38EF32F00A
:1067E0000401406B416B040120511F0B020A0FE0B2
:1067F000030A0BE0010A18E186D804014081020176
:10680000A7A112D0040140830FD07DD80DD050D85D
:1068100001E0010E5BD898C2E9FFEA6EEF50040B6D
:1068200003E00401010E406F020195050AE1020137
:10683000400E966F040E976F0201A7930201020E9D
:106840009A6F1200040122050EE120511F0B00096E
:106850000AE159D8030E0401215D03E10201A78179
:1068600002D00201A7910401225121E120511F0B06
:1068700002081DE124510F0B000919E019D801E0AD
:10688000010E24D8030E0401215D02E1840E03D021
:1068900024AF07D0400E98C2E9FF99C2EAFFEF6E1D
:1068A0001200880E98C2E9FF99C2EAFFEF6E12004B
:1068B0002ED80F0B080DF3500101CD6B000FCC6FDC
:1068C000040ECD2304012451800B1200040DF3505B
:1068D0000101CC250201986F000E0101CD210201BA
:1068E000996F120010D804012251F66EF76AD89001
:1068F000F636F7361200F7220900F5CF96F20A00B5
:10690000F5CF97F212000201010E956F1200FBDF26
:06691000040124511200F5
:0A691600D9CFE6FFDACFE6FFFA0E54
:10692000E3CFD9FFFB0EE3CFDAFFFC0EE3CFE9FFA5
:10693000FD0EE3CFEAFFE9CFF3FFEACFF4FFF80E55
:10694000E35003E1F90EE35008E0F80EE30602E23B
:10695000F90EE306DECFEEFFF2D7FF0EE3CFDAFF4C
:10696000E552FF0EE3CFD9FFE5521200FB0EE3CF55
:10697000F6FFFC0EE3CFF7FFFD0EE3CFF8FFFE0EB0
:10698000E3CFE9FFFF0EE3CFEAFFE9CFF3FFEACF62
:10699000F4FFF90EE35003E1FA0EE35009E0F90EBB
:1069A000E30602E2FA0EE3060900F5CFEEFFF1D7A7
:1069B0001200FE0EE3CFE9FFFF0EE3CFEAFFE9CFBF
:1069C000F3FFEACFF4FFFB0EE35003E1FC0EE350CC
:1069D00009E0FB0EE30602E2FC0EE306FD0EE350C7
:1069E000EE6EF1D71200D9CFE6FFDACFE6FFFA0E4E
:1069F000E3CFD9FFFB0EE3CFDAFFFC0EE3CFE9FFD5
:106A0000FD0EE3CFEAFFE9CFF3FFEACFF4FFEE6636
:106A1000FED7ED52DFCFEEFFDE66FCD7FF0EE3CFF1
:106A2000DAFFE552FF0EE3CFD9FFE5521200FB0E6D
:106A3000E3CFF6FFFC0EE3CFF7FFFD0EE3CFF8FF49
:106A4000FE0EE3CFE9FFFF0EE3CFEAFFE9CFF3FF4E
:106A5000EACFF4FFEE66FED7ED520900F5CFEFFF67
:106A6000EE66FBD71200FE0EE3CFE9FFFF0EE3CF89
:106A7000EAFFFD0EE350EF5C05E0EE66FAD7F36A3D
:106A8000F46A04D0E9CFF3FFEACFF4FF1200FB0E63
:106A9000E3CFF6FFFC0EE3CFF7FFFD0EE3CFF8FFE9
:106AA000FE0EE3CFE9FFFF0EE3CFEAFFE9CFF3FFEE
:106AB000EACFF4FF0900F5CFEFFFEE66FBD7120037
:106AC000FE0EE3CFE9FFFF0EE3CFEAFFF36AF46ABD
:106AD000EE5203E0F34AF42AFBD71200D9CFE6FFC7
:106AE000DACFE6FFFA0EE3CFD9FFFB0EE3CFDAFFF2
:106AF000FC0EE3CFE9FFFD0EE3CFEAFFF80EE35013
:106B000003E1F90EE3500AE0F80EE30602E2F90EA3
:106B1000E306DE50EF5C02E1EE66F0D7F36EFF0EA7
:106B2000E3CFDAFFE552FF0EE3CFD9FFE552F35092
:106B30001200D9CFE6FFDACFE6FFFA0EE3CFD9FF96
:106B4000FB0EE3CFDAFFFC0EE3CFE9FFFD0EE3CF50
:106B5000EAFFE9CFF3FFEACFF4FFF80EE35003E1D9
:106B6000F90EE3500BE0F80EE30602E2F90EE3063D
:106B7000DECFEFFFEE66F1D7DD52EFD7FF0EE3CFAA
:0E6B8000DAFFE552FF0EE3CFD9FFE552120017
:026B8E000BD822
:106B9000E552E5CFA5F2E5CFA4F2E5CFA3F2E7CF2A
:106BA000A2F248E8000C46E8D9CFE6FFDACFE6FFCC
:106BB000E1CFD9FFE2CFDAFF90E90A6A0B6A0C6AEB
:106BC0000D6A00500502F450086E01500402F450A2
:106BD0000826000E096A092200500602F350082612
:106BE000F4500922000E0A2201500502F350082633
:106BF000F4500922000E0A2202500402F350082623
:106C0000F4500922000E0A2200500702F350092610
:106C1000F4500A22000E0B2201500602F3500926FE
:106C2000F4500A22000E0B2202500502F3500926EE
:106C3000F4500A22000E0B2203500402F3500926DE
:106C4000F4500A22000E0B2201500702F3500A26CC
:106C5000F4500B22000E0C2202500602F3500A26BA
:106C6000F4500B22000E0C2203500502F3500A26AA
:106C7000F4500B22000E0C2202500702F3500B2698
:106C8000F4500C22000E0D2203500602F3500B2686
:106C9000F4500C22000E0D2203500702F3500C2674
:106CA000F4500D22000E0E2207AE06D000500A5EF0
:106CB00001500B5A02500C5A03AE06D004500A5E23
:106CC00005500B5A06500C5A89EB00F08AEB01F084
:106CD0008BEB02F08CEB03F0E552E5CFDAFFE7CF68
:106CE000D9FF4AE9000C0AD844E9E6CFA2F2E6CF80
:106CF000A3F2E6CFA4F2E6CFA5F2000C46E8D9CF86
:106D0000E6FFDACFE6FFE1CFD9FFE2CFDAFF8CE989
:106D100044E8036624D082EB09F0010E0F6E200ECA
:106D20000E6E0D6A0C6A010E076E800E066E056A05
:106D3000046A040E086E09361FE2093609E384EB83
:106D40000CF085EB0DF086EB0EF087EB0FF014D016
:106D5000D8900E360F3606360736082EECD7660E5C
:106D600083EB09F0094ECD0E094EA60E094E880E92
:106D70000E6E0C6A0D6A0F6A080E0201B567B551F6
:106D8000086E0CEBE6FF0DEBE6FF0EEBE6FF0FEBFC
:106D9000E6FF00EBE6FF01EBE6FF02EBE6FF03EBAD
:106DA000E6FF0CEBE6FF0DEBE6FF0EEBE6FF0FEB6D
:106DB000E6FFD3EC35F0D3EC35F0000ED88010565A
:106DC00011561256030E1356D3EC35F0D8900F32ED
:106DD0000E320D320C32082ED4D7E552E550036E38
:106DE000E550026EE550016EE750006EE552E5CFCA
:0A6DF000DAFFE7CFD9FF46E9000CF7
:066DFA00ECD883E901342E
:106E00000AE300EBCCF101EBCDF10101CC6DCD1F1C
:106E1000000ECD2304D000EBCCF101EBCDF1CCC1C1
:106E2000F3FFCDC1F4FF41E9E7CFD9FF1200D2D87B
:106E300086E949E8C9D800EBE6FF01EBE6FFCDECB7
:106E400038F044E9C1D860EC35F042E9F3500E6EF9
:106E50000E50025C0E6E0E3401E30E6A0E50025CA0
:106E60000101CC6FCD6B800B01E0CD69CCC1E6FF99
:106E7000CDC1E6FFA9D80EEBD0F1D16BD0BFD1695F
:106E80000350D025CE6F0450D121CF6FCEC1E6FF85
:106E9000E66E8BEC34F046E94AE9E7CFD9FF120001
:106EA00099D886E9013402E32D0E01D02B0EE66E4F
:106EB00003EBE9FF04EBEAFFE552E750EF6E00EB6E
:106EC000E6FF01EBE6FF99DF42E9F3CFE6FFF4CFFF
:106ED000E6FF02EBE6FF03EBE6FF04EBE6FFA7DFCE
:106EE00045E941E9E7CFD9FF120074D887E941E8C5
:106EF000076A03340350071802E60350075C36E2C2
:106F000003EBD0F10101D16BD0BFD1693FD8D2BF23
:106F1000D36965D8EF380F0BF66EF76AF6BEF768DF
:106F200049D8CC6FCD6B800B01E0CD693CD8E552E0
:106F3000E750EF6E03EBD0F1D16BD0BFD16926D80B
:106F4000D2BFD3694CD8EF500F0BF66EF76AF6BE7E
:106F5000F76830D8010FCC6FCD6B800B01E0CD69A5
:106F600022D8E552E750EF6E072AC3D700500AE057
:106F70000750E8240101CC6FCD6B800B01E0CD6997
:106F800012D8EF6A42E9E7CFD9FF12000150D025AD
:106F9000CE6F0250D121CF6FCE07000ECF5B07EB33
:106FA000D2F1D36B1200CC510424E96ECD510520EF
:106FB000EA6E1200200EF6267F0EF7220800F5502A
:106FC000E66E0750E8241200D950060FE66EDACFBD
:106FD000E6FF1200D9CFE6FFE1CFD9FF1200D25170
:0C6FE000CE5DE96ECF51D355EA6E120071
:046FEC0081B804D094
:106FF0006DB604D00FD802D06DB613D80201A60525
:1070000008E16DBA06D0686A696A69806988020E0B
:10701000A66F12006D6A696A6D860201010EA66F85
:1070200012006D6A696A0201A66B120011EF38F056
:107030000201A65101E112006850040B04E06950FE
:10704000040B01E045D86DB212006850010B04E05A
:107050006950010B01E069D86850100B04E06950D9
:10706000100B01E02ED86850400B04E06950400B33
:1070700001E047D86850200B04E06950200B01E084
:1070800042D86850020B04E06950020B01E04BD873
:10709000030E0201A65D01E212000201AE6B040EB6
:1070A000AE5D0EE26850080B0BE06950080B08E07B
:1070B00065EC30F0000901E168960201AE2BEFD7D4
:1070C0001200698468986D82A19AA08AA09A120021
:1070D0006D92699468A402D06894FCD712000201F2
:1070E000A7A10ED06D926D840201080EAF6F070E3E
:1070F000B06FAF07000EB05BAF51B011FAE16D9405
:107100001200689C120070A00CD0800E0401005D7B
:1071100007E1840E0401045D03E104018C0E006F9D
:107120007090689A12006A6A12006A6A686A9F0E12
:107130006B6E7B0E696E6E6A0F0EE66E710EE66EFA
:107140000F0EE66E18D843E9160E706E68A608D0CA
:107150006896000000000000000000000000F6D764
:107160006D987CEC31F00201A7910201A86B02013D
:10717000030EA66F1200D9CFE6FFE1CFD9FF84E955
:1071800001EBE9FF02EBEAFF005003E0EE6A0006C4
:0A719000FBD741E9E7CFD9FF120059
:06719A00D9CFE6FFDACFB9
:1071A000E6FFFA0EE3CFD9FFFB0EE3CFDAFFFD0EC9
:1071B000E35209E72D0EDE6EFC0EE31EE32AFD0E00
:1071C000D8B4E306E31EE652E652E652FD0EE12491
:1071D000E76EFF0EE220E46EE652F70EE3CFE6FF25
:1071E000F70EE3CFE6FF3DEC39F0F90EE124E96E4E
:1071F000FF0EE220EA6E2DEC39F00AE12AEC39F0BC
:1072000009E12DEC39F008E12AEC39F007E108D06A
:1072100038EC39F033EC39F038EC39F033EC39F044
:1072200038EC39F0DE6AF90EE126FF0EE222FF0E9D
:10723000E3CFDAFFE552FF0EE3CFD9FFE552FC0EB4
:10724000E124E96EFF0EE220EA6EEECFF3FFEFCF0E
:10725000F4FF1200EF380F0B1200EF500F0B02E19A
:10726000EE52D8841200EF380F0B300FDE6E120092
:10727000EE500F0B300FDE6E1200FC0EE3CFE9FF75
:10728000FD0EE3CFEAFF100EE66EEE6AEE6AEF6ADD
:10729000D890FD0EE336FE0EE336ED36ED36EF36D2
:1072A000FF0EE30609E05EEC39F0EE525EEC39F0D9
:1072B000EE525EEC39F0EDD7E56E1200030EEF24CE
:0E72C000E8B6EF6E300EEF24E8BEEF6E000C65
:0272CE000000BE
:1072D000000000005F00000000030003000006093A
:1072E0000906242A7F2A122313086462364956208D
:1072F00050000B07000000003E410000413E00002E
:10730000082A1C2A0808083E080800583800000807
:1073100008080808003030000020100804023E5120
:1073200049453E00427F4000625149494622414959
:1073300049361814127F1027454545393C4A4949BA
:107340003001710905033649494936064949291E64
:107350000036360000005B3B000000081422411498
:1073600014141414412214080002015109063E416C
:107370005D551E7E0909097E7E494949363E4141D7
:1073800041227F4141413E7F494949417F090909E5
:10739000013E414151327F0808087F00417F410092
:1073A000204040403F7F081422417F404040407FC2
:1073B000020C027F7F0408107F3E4141413E7F095D
:1073C0000909063E4151215E7F091929462649498E
:1073D000493201017F01013F4040403F07186018DA
:1073E000077F2018207F63140814630304780403C4
:0573F000615149454315
:0B73F5003030303020303030300030BD
:107400003030330030303020303030005858585849
:10741000585858582058585858585858582058585C
:10742000585858585858004869796100455258587A
:1074300000434C5858004C303030004D3030300054
:10744000484F4C4400534156450052415720004894
:1074500049474800475241440043414C20002030F6
:107460003023005341502000303030250048454C37
:107470005000303030300030303047004330303052
:107480000030303023002A20200D0A0024505450B0
:10749000534854442C003030303030300041545A7E
:1074A0000A0041542B42545343414E2C332C300A92
:1074B0000041542B42544D4F44452C330A00415453
:1074C0002B42544E414D453D22536865746C616EAC
:1074D000642041747461636B20506F6E79222F6E4B
:0774E0000041545A2F6E0019
:0974E7001201000202000020D88D
:1074F000040A000000010200010902430002010029
:10750000803209040000010202010005240010017C
:1075100004240202052406000105240100010705D8
:10752000820308000209040100020A0000000705A6
:107530000302400000070583024000000403090421
:10754000340355006E0064006500720077006F0020
:107550006F006400200055006E006400650072003A
:10756000670072006F0075006E006400200020004C
:1075700020002000340353006800650074006C0094
:1075800061006E006400200041007400740061001E
:1075900063006B00200050006F006E007900200037
:1075A0002000200020002000F974F9743C7540751B
:0475B0007475CC63BF
:0C75B4002A0EF66E080EF76E000EF86E40
:1075C00002010900F5508F6F0900F550906F03E13B
:1075D0008F6701D03DD00900F5508A6F0900F55042
:1075E0008B6F0900F5508C6F09000900F550E96EAA
:1075F0000900F550EA6E090009000900F5508D6F89
:107600000900F5508E6F09000900F6CF91F2F7CF0F
:1076100092F2F8CF93F28AC2F6FF8BC2F7FF8CC2C8
:10762000F8FF02018D5302E18E5307E00900F55087
:10763000EE6E8D07F8E28E07F9D791C2F6FF92C27F
:10764000F7FF93C2F8FF02018F07000E905BBFD7D0
:02765000120026
:0E765200D9CFE6FFDACFE6FFE1CFD9FFE2CFD6
:10766000DAFF87E9A0EC3FF0C580C5B0FED7A1B630
:107670002CD004EBE6FF35D80FE1C5BC28D003EBD6
:10768000E6FF2FD809E1C5BC22D0C582C5B2FED71E
:107690000428E66E26D803E0C584FD0E1CD0C5BCC8
:1076A00016D000EBE6FF01EBE6FF02EBE6FF5DEC38
:1076B0003DF043E9000909E1C58AC588C5B8FED790
:1076C000C584C5B4FED7A1A605D0FF0E04D0C584DD
:1076D000FE0E01D0000E41E9E5CFDAFFE7CFD9FF7A
:0C76E0001200B1EC3DF041E9000912007D
:0476EC00D9CFE6FF0D
:1076F000DACFE6FFE1CFD9FFE2CFDAFF84E9A0ECF1
:107700003FF0C580C5B0FED7A1B626D001EBE6FF9D
:1077100033D811E1C5BC22D000EBE6FF2DD80BE138
:10772000C5BC1CD0C582C5B2FED7A1B615D00128F4
:10773000E66E22D803E0C584FD0E12D0C5BC0ED083
:10774000C586C5B6FED7C58AC588C5B8FED7C58467
:10775000C5B4FED7A1A607D0F36803D0C584FE0E3A
:10776000F36EF46803D0C950F36EF46A41E9E5CFD3
:10777000DAFFE7CFD9FF1200B1EC3DF041E9000993
:027780001200F5
:0E778200D9CFE6FFDACFE6FFE1CFD9FFE2CFA5
:10779000DAFF85E9AC6AAB6A02B0AC8802A202D01B
:1077A000AC8CAB8C02B4AC8E02A602D0AB8801D0FC
:1077B000AB8A02B8AC849E9802BAAB8602AC02D007
:1077C0009D8A01D09D9A9E9A02AE02D09D8801D0DA
:1077D0009D9800EBAFFF010101EBCCF1CD6BCCC16B
:1077E000B0FFAC8AAB8E949C948EAC50100B04E02E
:1077F000AC50800B01E1948C41E9E5CFDAFFE7CF93
:04780000D9FF12009A
:0C780400D9CFE6FFDACFE6FFE1CFD9FFD5
:10781000E2CFDAFF85E9A0EC3FF0C580C5B0FED726
:10782000A1B61BD002EBE6FF21D80CE1C5BC0DD000
:1078300001EBE6FF1BD806E1C5BC07D000EBE6FF75
:1078400015D806E0C584FD0E0BD0C584FE0E08D009
:10785000C584C5B4FED7A1A602D0FF0E01D0000E8C
:1078600041E9E5CFDAFFE7CFD9FF1200B1EC3DF0F7
:0678700041E900091200CD
:0A7876000000000000000000000008
:1078800000000000000000000000000000000000F8
:1078900000000000000000000000000000000000E8
:1078A00000000000000000000000000000000000D8
:1078B00000000000000000000000000000000000C8
:1078C00000000000000000000000000000000000B8
:0E78D0000000000000000000000000000000AA
:0278DE00F36A4B
:1078E000F46AFF0EE124E96EFF0EE220EA6EED6617
:1078F00013D02F0EEF6410D0390EEF640CD0400E71
:10790000EF640AD05A0EEF6406D0600EEF6404D024
:107910007B0EEF6001D0F32A1200F36AF46AFF0EC7
:10792000E124E96EFF0EE220EA6EED660AD0200E39
:10793000EF5C06E0080EEF6404D00E0EEF6001D09D
:04794000F32A120014
:0C794400D9CFE6FFE1CFD9FF82E941E88E
:10795000080E026E00EBB2F28B940201B2BF8B8470
:1079600000000000D8908BB4D8808B90B237000014
:107970000000000000000000000000000000000007
:10798000000000008B808B940201B2BF8B84020642
:107990000250E8E10201B25100D042E9E7CFD9FF3D
:0279A0001200D3
:0E79A200D9CFE6FFDACFE6FFE1CFD9FFE2CF83
:1079B000DAFF83E944E8F8CF05F0F6CF06F00C0EC5
:1079C000BA6E050EF66EF76A300EF86E0800F550C6
:1079D000010B02E0046801D0046A045002E09492B2
:1079E00001D09396CA9400EBCBFFCA8405C0F8FF80
:1079F00006C0F6FF45E9E5CFDAFFE7CFD9FF120071
:107A0000D9CFE6FFDACFE6FFE1CFD9FFE2CFDAFF49
:107A100085E9C26AC06A01407F0B3C0BC26E013827
:107A2000F00B300B0010C16E0250040DF350380BF8
:107A30000101CD6F02380F0B070BCC6F800E0214C3
:107A4000CC11CD11C06E01AE03D09E9C9D8CF28CEA
:0E7A5000C28041E9E5CFDAFFE7CFD9FF12008F
:027A5E00D9CF7E
:107A6000E6FFDACFE6FFE1CFD9FFE2CFDAFF85E923
:107A7000ACA2FED700EBF6FF01EBF7FF02EBF8FF3D
:107A80000800F5CFE6FF34EC3FF041E9D9CFE9FF3C
:107A9000DACFEAFFEFCFF6FFEE2AEFCFF7FF000EC7
:107AA000EE22EFCFF8FFEE220800F550E1E141E9C8
:0A7AB000E5CFDAFFE7CFD9FF12009F
:067ABA00D9CFE6FFDACF90
:107AC000E6FFE1CFD9FFE2CFDAFF85E900500006FB
:107AD00000091AE0B3EC3FF0E66E01EBE9FF02EBC0
:107AE000EAFF012A000E0222E552E750EF6EC5B60A
:107AF000FED7A1A602D0FF0E08D00050E7E0C59A3D
:107B0000C588C5A8E3D7FDD7000E41E9E5CFDAFF68
:067B1000E7CFD9FF1200CF
:0A7B1600D9CFE6FFDACFE6FFE1CF9A
:107B2000D9FFE2CFDAFF84E942E880EB04F081EB91
:107B300005F0060ED89004360536E804FBE105EBA7
:107B4000BBFF0440E8423F0B300B0101CC6FCF0E6E
:107B5000BA14CC11BA6E43E9E5CFDAFFE7CFD9FF0B
:027B6000120011
:0E7B6200D9CFE6FFDACFE6FFE1CFD9FFE2CFC1
:107B7000DAFF83E900EBC9FFC6AE02D0FF0E11D0D9
:107B8000C7B0FED70F0EC614080804E00F0EC614C7
:107B9000090802E1A0EC3FF0C5AC02D0FE0E01D016
:0E7BA000000E41E9E5CFDAFFE7CFD9FF120072
:027BAE00D9CF2D
:107BB000E6FFDACFE6FFE1CFD9FFE2CFDAFF84E9D3
:107BC000ACA2FED700EBE9FF01EBEAFFEFCFE6FF47
:107BD00034EC3FF041E900EBE9FF01EBEAFF002A5A
:107BE000000E0122EF50ECE141E9E5CFDAFFE7CFEB
:047BF000D9FF1200A7
:0C7BF400D9CFE6FFDACFE6FFE1CFD9FFE2
:107C0000E2CFDAFF83E9360E0014B16EB36AB26ACE
:107C1000A19200AE02D0A08201D0A09200A002D01A
:107C2000B18E01D0B19EB18041E9E5CFDAFFE7CF57
:047C3000D9FF120066
:0C7C3400D9CFE6FFDACFE6FFE1CFD9FFA1
:107C4000E2CFDAFF83E97E0E0014CD6E00AC02D0E5
:107C5000CD8E01D0CD9ECF6ACE6A9E9000AE02D06E
:107C60009D8001D09D90CD8041E9E5CFDAFFE7CF3F
:047C7000D9FF120026
:0C7C7400FF0EE3500201B16FEE0E02D0D3
:107C8000F20E0000E76EE72E43EF3EF00C0E01010E
:107C9000FF6FE76AE72E4AEF3EF0FF2F49EF3EF015
:0A7CA0000201B12F40EF3EF0120088
:067CAA00D9CFE6FFDACF9E
:107CB000E6FFE1CFD9FFE2CFDAFF83E97F0E0014C0
:107CC000D56ED76AD66AF29400AE02D0F28A01D09D
:107CD000F29AD58E41E9E5CFDAFFE7CFD9FF12005E
:107CE000D9CFE6FFDACFE6FFE1CFD9FFE2CFDAFF67
:107CF00083E9FB0E0014CA6ECC6A9E9200AE02D0DD
:107D00009D8201D09D92CA8441E9E5CFDAFFE7CF99
:047D1000D9FF120085
:0C7D1400D9CFE6FFDACFE6FFE1CFD9FFC0
:107D2000E2CFDAFF84E93F0EC716C66AC56A015082
:107D3000C6120050C71293829380C68A41E9E5CFEC
:087D4000DAFFE7CFD9FF1200C2
:087D4800D9CFE6FFDACFE6FF18
:107D5000E1CFD9FFE2CFDAFF84E942E880EB04F01B
:107D600081EB05F005EBB3FF04EBB2FF43E9E5CF90
:087D7000DAFFE7CFD9FF120092
:087D7800D9CFE6FFDACFE6FFE8
:107D8000E1CFD9FFE2CFDAFF82E942E8B250026EDA
:107D9000B350036E02EBF3FF03EBF4FF43E9E5CFCF
:087DA000DAFFE7CFD9FF120062
:087DA800D9CFE6FFDACFE6FFB8
:107DB000E1CFD9FFE2CFDAFF84E942E880EB04F0BB
:107DC00081EB05F005EBCFFF04EBCEFF43E9E5CFF8
:087DD000DAFFE7CFD9FF120032
:087DD800D9CFE6FFDACFE6FF88
:107DE000E1CFD9FFE2CFDAFF82E942E8CE50026E5E
:107DF000CF50036E02EBF3FF03EBF4FF43E9E5CF53
:087E0000DAFFE7CFD9FF120001
:087E0800D9CFE6FFDACFE6FF57
:107E1000E1CFD9FFE2CFDAFF84E942E880EB04F05A
:107E200081EB05F005EBD7FF04EBD6FF43E9E5CF87
:087E3000DAFFE7CFD9FF1200D1
:087E3800D9CFE6FFDACFE6FF27
:107E4000E1CFD9FFE2CFDAFF82E942E8D650026EF5
:107E5000D750036E02EBF3FF03EBF4FF43E9E5CFEA
:087E6000DAFFE7CFD9FF1200A1
:087E6800D9CFE6FFDACFE6FFF7
:107E7000E1CFD9FFE2CFDAFF83E9ACAC04D0AC901C
:107E80000201B3B3AC8000EBADFF41E9E5CFDAFF0F
:067E9000E7CFD9FF12004C
:0A7E9600D9CFE6FFDACFE6FFE1CF17
:107EA000D9FFE2CFDAFF83E900EBB8FF41E9E5CF84
:087EB000DAFFE7CFD9FF120051
:087EB800FF0EE3500201B16F5F
:107EC0001A0E00D000D001D0200EE76EE72EFED7AC
:087ED000B12FFAD700D0120017
:087ED80013EE00F023EE00F0B0
:107EE000F86ADAEC3AF0CBEC3FF0CFEC04F0FBD7D9
:027EF00012007E
:0E7EF200C4CFCEF1CEC1CFF10101CE6BC35093
:0A7F0000CE11F36ECFC1F4FF1200A2
:067F0A00FF0EE350E84EFB
:107F10001200000000D000D000D0E82EFAD71200E6
:107F200030313233343536373839414243444546AF
:017F30000050
:017F3100004F
:0E7F3200898A8B948B80929A9494949012007A
:0E7F40001F0EC514FDE1C750040BFAE112003C
:027F4E0000EE43
:0C7F500000F00F0EEE6AEA62FDD712008E
:047F5C000A4F4B0A73
:067F6000000A4B4F0A006D
:0A7F6600C586C7A0FED7C95012005F
:0A7F7000C250020B01E0010E1200E6
:067F7A00B190A09212007C
:067F8000C2909D9C12005E
:047F8600898A1200D2
:047F8A00C69A120081
:027F8E00899ACE
:027F90001200DD
:047F9200C282120095
:027F96001200D7
:047F98003D0A270077
:047F9C00C7711C018C
:097FA0000000000A0000010000CD
:067FA900FF0101FFFF01D2
:017FAF0003CE
:0C7FB000B84B390049920400000040006A
:020000040030CA
:0100000038C7
:010001000EF0
:010002001CE1
:010003001CE0
:01000500807A
:01000600C138
:010008000FE8
:01000900C036
:01000A000FE6
:01000B00E014
:01000C000FE4
:01000D0040B2
:0200000400F00A
:0100FF00AA56
:00000001FF
